:020000040000FA
:06000000E3EF35F01200F1
:0600080097EF2FF012003B
:06002A0006005E6C000000
:1000300075030000040000003C6C00009602000004
:1000400022000000146C00006E0200002800000076
:10005000126C0000FD01000002000000106C0000A6
:10006000FE00000002000000006C00002D030000F4
:04007000100000007C
:0C0074000901006B0A0E005D26E200513D
:10008000220DF3CF01F9F4CF02F9000E01270A0E79
:100090000223DFEC08F0EF6A34EC0AF0EF9034EC66
:1000A0000AF0EF8234EC0AF0EF8434EC0AF0EF98B7
:1000B00034EC0AF0EF96DFEC08F0EFEC09F0DFEC3F
:1000C00008F003EC0AF0002BD7D70101496B040EAE
:1000D0004A6F4B6B4C6B4D6B4E6B12000901006B02
:1000E0000A0E005D36E20051220DF3CF01F9F4CF84
:1000F00002F9000E01270A0E0223CEEC08F0EF50A1
:10010000000925E1CEEC08F0010EEF6ECEEC08F010
:100110000B0E4FC1EBFF0C0E50C1EBFFCEEC08F005
:100120000D0EEB6A0E0EEB6ACEEC08F0FFEC09F058
:1001300046EC0AF0EF8046EC0AF0EF96CEEC08F0C1
:10014000EFEC09F046EC0AF0EF8200511200002BB0
:10015000C7D7FE0C09016F6B6C6B0A0E6C5D14E265
:100160006C51220DF3CF6DF9F4CF6EF9000E6D27AF
:100170000A0E6E2385EC08F0EF50000903E1010E32
:100180006F6F02D06C2BE9D76F5101E1FE0C0101BA
:10019000492B000E4A2385EC08F00B0E49C1EBFFFA
:1001A0000C0E4AC1EBFF880ED8804955130E4A55F4
:1001B00003E2496B040E4A6F85EC08F0A1EC09F0EC
:1001C000EF9085EC08F00D0E53C1EBFF0E0E54C1FD
:1001D000EBFF4B2B000E4C234D234E2307EC0AF074
:1001E00043EC09F085EC08F0180E6DEC08F067ECB4
:1001F00009F00A0EE66EE66A51C1E6FF52C1E6FF5B
:1002000085EC08F08FEC08F0F9EC08F00101020E23
:100210007E6F85EC08F0F3EC09F007EC0AF0E9ECEE
:1002200008F085EC08F0F7EC09F085EC08F0FBEC41
:1002300009F085EC08F0D8EC08F085EC08F0030E26
:10024000EF6E07EC0AF093EC09F085EC08F0F2ECA5
:1002500008F009016C51120001015551A8EC08F099
:10026000EF50040801E0000C010C01015651220D71
:10027000F3CF81F9F4CF82F9000E090181270A0E2C
:100280008223E4EC08F0EF50040806E081C988F10D
:1002900082C989F1CCEF06F056C160F14CD9F9EC76
:1002A00008F00101110E7E6FE4EC08F0F3EC09F0A8
:1002B000E4EC08F037EC0AF0E9EC08F0E4EC08F0C4
:1002C000F7EC09F0E4EC08F0FBEC09F0E4EC08F0E2
:1002D000D8EC08F0E4EC08F037EC0AF093EC09F005
:1002E000E4EC08F0050EEF6E120001015751220DEB
:1002F000F3CF83F9F4CF84F9000E090183270A0EA6
:1003000084238AEC08F09DEC09F001E1000C8AECF2
:1003100008F023EC0AF0020B01E1000C8AEC08F073
:10032000100E6DEC08F0EECF80F1EDCF81F18AEC8C
:1003300008F00F0EEB5001017F6F0101100E7E6F70
:10034000F3EC09F08AEC08F037EC0AF0E9EC08F07D
:100350008AEC08F0F7EC09F08AEC08F0FBEC09F005
:100360008AEC08F0D8EC08F08AEC08F0100EC8EC23
:1003700009F0126A136A8AEC08F037EC0AF01050A0
:10038000EE261150EE221250EE221350EE2255ECC2
:100390000AF0EF9255EC0AF0EF988AEC08F022ECA4
:1003A00009F08AEC08F0EFEC09F055EC0AF0EF8266
:1003B000010C0A0E0101585D13E25851A8EC08F037
:1003C0000F0E6DEC08F0EF50FF0802E14CEF0BF060
:1003D0005851A8EC08F023EC0AF0020B02E0010CE3
:1003E000000E120001015951220DF3CF81F9F4CF13
:1003F00082F9000E090181270A0E8223D3EC08F04E
:100400009DEC09F014E1D3EC08F00F0E1BC0EBFFDC
:10041000D3EC08F0EB500201596F89EC0DF0D3ECEE
:1004200008F04CEC09F0D3EC08F07BEC09F0D3ECCD
:1004300008F026EC0AF001E3000CD3EC08F0A1EC84
:1004400009F0EF885AC150F25CEC0BF0D3EC08F0E5
:10045000100E6DEC08F0EE2AEF22D3EC08F026EC3B
:100460000AF003E359C157F140DF010C01015B5170
:10047000220DF3CF6CF9F4CF6DF9000E09016C2752
:100480000A0E6D23B7EC08F09DEC09F014E1B7EC0F
:1004900008F00F0E1BC0EBFFB7EC08F0EB500201A9
:1004A000596F89EC0DF0B7EC08F04CEC09F0B7ECA3
:1004B00008F07BEC09F0B7EC08F026EC0AF001E359
:1004C000000C0DEC0AF0EE24106E5F51EE20116E60
:1004D000CA0ED8801054030E11540EE2B7EC08F087
:1004E000100E6DEC08F0EECF5EF1EFCF5FF1CA0EAB
:1004F000D8805E57030E5F57B7EC08F0A1EC09F007
:10050000EF885EC153F25FC154F25CC151F25DC12C
:1005100052F29CEC0BF00DEC0AF0EE265F51ED224E
:10052000B7EC08F026EC0AF003E35BC157F1DDDE1F
:1005300001015E51120001016051220DF3CF00F95B
:10054000F4CF01F9000E090100270A0E012300C9AA
:10055000E9FF01C9EAFF52EC0AF001E1000C97EC57
:100560000DF000C9E9FF01C9EAFFA1EC09F0EF961F
:10057000010C01016151220DF3CF20F9F4CF21F9D3
:10058000000E090120270A0E212318EC09F052EC75
:100590000AF02BE018EC09F023EC0AF0040B08E059
:1005A000280E1DEC09F018EC09F0A1EC09F0EF940D
:1005B00018EC09F04CEC0AF0EE50ED1008E197EC65
:1005C0000DF018EC09F0A1EC09F0EF96000C18EC16
:1005D00009F04CEC0AF0EE06EF5AC4EC0CF062C1E4
:1005E000E9FF63C1EAFFEF6E010C000C01016451E9
:1005F000220DF3CF02F9F4CF03F9000E090102270F
:100600000A0E0323FFEC08F052EC0AF03AE0FFEC8C
:1006100008F023EC0AF0040B08E0280E1DEC09F0AA
:10062000FFEC08F0A1EC09F0EF94FFEC08F0120EDB
:10063000C8EC09F001016751105C6851115808E2DB
:10064000FFEC08F04CEC0AF0EECF67F1EDCF68F16B
:10065000FFEC08F04CEC0AF0EE50ED1008E197ECDE
:100660000DF0FFEC08F0A1EC09F0EF960AD067C19D
:1006700057F268C158F265C155F266C156F227EFCC
:100680000DF0F36AF46A12000A0E0101695D07E2D7
:100690006951A8EC08F052EC0AF002E0010C000EDF
:1006A00012000901736B6C6B0A0E6C5D01E3D4D010
:1006B0006C51220DF3CF6DF9F4CF6EF9000E6D275A
:1006C0000A0E6E237BEC08F052EC0AF001E0C1D078
:1006D0007BEC08F023EC0AF0100B01E0BAD07BECC5
:1006E00008F0EF50000901E1B4D07BEC08F0EF50C6
:1006F000010807E17BEC08F023EC0AF0010B01E0B4
:10070000A8D07BEC08F01D0E6DEC08F00301EE5054
:10071000645D106EEE506559116E7BEC08F01F0E93
:100720006DEC08F071EC09F01050125C1150135888
:1007300001E38FD04CEC0BF0000901E112007BECDF
:1007400008F0F2EC08F07BEC08F01F0E6DEC08F0FE
:10075000EE2AEF227BEC08F01C0E6DEC08F0EF2A7D
:100760007BEC08F0EF50060A27E0010A25E0020AB8
:100770001CE00F0A1AE00E0A10E0060A05E0010A62
:1007800028E10901020E24D013EC0AF0106E030ECA
:10079000105C16E20901120E1BD00901110E736FD5
:1007A0007BEC08F0050EEF6E14D013EC0AF0030892
:1007B00007E30901010E0CD013EC0AF0030806E26E
:1007C0006DC988F16EC989F1E7DA03D00901100E0D
:1007D000736F0901735100083CE2100E735D11E064
:1007E0007BEC08F037EC0AF0EFCF6FF9EE2AEFCF91
:1007F00070F9EE22EFCF71F9EE22EFCF72F9EF220E
:100800000CD07BEC08F037EC0AF0EECF6FF9EECFAE
:1008100070F9EECF71F9EFCF72F9F9EC08F073C906
:100820007EF17BEC08F0F3EC09F06FC976F170C94A
:1008300077F171C978F172C979F17BEC08F0F7ECC6
:1008400009F07BEC08F0FBEC09F07BEC08F0D8EC4D
:1008500008F009016C2B28D71200140E0201576F03
:10086000586B02016C0E556F090E566F27EC0DF098
:1008700001016C0E866F090E876F59DA6AC1E9FFB4
:100880006BC1EAFF4FEC0AF0EECF80F9EECF81F9B1
:10089000EECF82F9EFCF83F998EC09F0EFCF84F92E
:1008A000010E6DEC08F0EFCF85F998EC09F0020E1F
:1008B0006DEC08F0EFCF86F998EC09F0030E6DECC3
:1008C00008F0EFCF87F90901886B060E896F6EC1BA
:1008D0008AF96FC18BF96EC1D8F26FC1D9F28BEC76
:1008E00025F0F3CF8AF9F4CF8BF90C0E0201E06FFB
:1008F000E16B0201800EDE6F090EDF6FBFEC25F0A9
:10090000F3CF8DF9F4CF8EF909018D1F8E1F240EC0
:100910001DEC09F08DC950F25CEC0BF08EC950F261
:100920005CEC0BF0140E1DEC09F06EC1E2F26FC12D
:10093000E3F21BEC26F0F3CF8DF9F4CF8EF9090129
:100940007C51F31802E17D518E1903E097EC0DF014
:10095000010C55EC09F0106E116A140E105E000EB9
:10096000115A10C08FF91050106E116AE850010131
:100970006E5D6E6F11506F596F6F140E6E5F000ECB
:100980006F5B090155EC09F00201696F6A6B140E87
:100990006927000E6A233DEC0FF06AC184F16BC138
:1009A00085F101016C0E826F090E836F3ED909013A
:1009B0008C6FFE0E8C5D11E26EC18FF16FC190F1F4
:1009C00001016C0E8D6F090E8E6F6AC18BF16BC1C8
:1009D0008CF18CC98AF106DA010C97EC0DF0FF0E50
:1009E00009018C5D37E101016E5109017427010194
:1009F0006F5109017523000E762377237951020B7D
:100A000003E17951010B05E0742B000E7523762369
:100A10007723EFDB0101040E7E6F70C97AF171C993
:100A20007BF172C97CF173C97DF174C976F175C926
:100A300077F176C978F177C979F16CC974F16DC92C
:100A400075F16EC972F16FC973F16AC170F16BC152
:100A500071F101D8010C72C148F973C149F974C12F
:100A60004AF975C14BF976C14CF977C14DF978C196
:100A70004EF979C14FF97AC150F97BC151F97CC166
:100A800052F97DC153F909015491549354955497E7
:100A90007EC155F9AAEC0DF0F3CF56F9F4CF57F912
:100AA0000901000EF35C040EF45804E3566B040EC7
:100AB000576F0DD0360ED8805655000E575505E2AB
:100AC000360E565F000E575B02D0566B576B586B55
:100AD000596B5A6B5B6B0101480E866F090E876F6D
:100AE00026D9140E01018027000E81237EA30ED08B
:100AF000040E8027000E81230901020E5C6F040E94
:100B00005D6F5E6F5F6B5499548B03D009015489FC
:100B1000549B548D549FB8C260F9B9C261F9BAC2EE
:100B200062F9BBC263F970C1E9FF71C1EAFF4FEC22
:100B30000AF0EECF64F9EECF65F9EECF66F9EFCFAC
:100B400067F9686B060E696F80C16AF981C16BF93C
:100B500080C1D8F281C1D9F28BEC25F0F3CF6AF9CC
:100B6000F4CF6BF90C0E0201E06FE16B0201600E35
:100B7000DE6F090EDF6FBFEC25F0F3CF58F9F4CF2D
:100B800059F90901581F591F58C946F959C947F958
:100B9000FF0E01017F5D02E11BC07FF1140E41DBFE
:100BA00080C157F381C158F30301060E566F70C11F
:100BB00054F371C155F3F6EC27F0140E0201536F94
:100BC000546B0201480E516F090E526F9CEC0BF0F2
:100BD00001017EA30BD0040E0201536F546B02017E
:100BE0005C0E516F090E526F9CEC0BF0140E19DB6A
:100BF00080C1E2F281C1E3F21BEC26F0F3CF46F9AB
:100C0000F4CF47F9240E0DDB47C950F25CEC0BF032
:100C100046C950F25CEC0BF002016C6B6D6B7FC14E
:100C20006BF250EC0FF0E6EF0EF00901FE0E036FD1
:100C3000026B0A0E025D4AE202511BDB84DAEF50BE
:100C4000000941E080DA0B0EA3DB50DB020E45DA2F
:100C500048DB00011250101836E11350111833E12F
:100C600072DAEF50010802E102C903F96CDA0D0EE5
:100C70008FDB3CDB36DB1250101825E113501118C6
:100C800022E184C1E9FF85C1EAFF4FEC0AF0EECF13
:100C900014F0EECF15F0EECF16F0EFCF17F053DAD9
:100CA000EE524FEC0AF0EE5014180DE1EE5015180C
:100CB0000AE1EE50161807E1EE50171804E103E1BF
:100CC0000901025112000901022BB3D70351D1DAF5
:100CD000FE0E035D27E037DAEF50010823E10A0E2C
:100CE000E66EE66A84C1E6FF85C1E6FF2CDA17DA14
:100CF0001250FCDA020E4CDB26DA0B0E10C0EBFFB2
:100D00000C0E11C0EBFFF2DA2DDA1DDAFADA1BDA7B
:100D100018DBEF9618DA63DB16DA13DBEF820901D2
:100D200003511200FE0E035D01E1FF0CFE0CDED943
:100D3000EFCF07F9A2DBE552E750EF6ED7D92BDBF7
:100D4000020E35DB020E09DB020E2BDB020EA1DBED
:100D5000040E09DB040E30DB080E05DB080E2CDB6D
:100D60000E0E25DB0E0EF9DA0E0E1BDB0E0E91DBDE
:100D7000100E1DDB100EF1DA100E13DB100E89DBE6
:100D8000120E15DB120EE9DA120E0BDB85DB010EFB
:100D9000A4D907C9EFFF1200D1D9CFDA06E0CED926
:100DA00051DACCD91CDB84DBEF82C8D928DBC6D969
:100DB0000D0EEB6A0E0EEB6AC1D974DB02E097EC04
:100DC0000DF076DBEF96BAD91EDB72DBEF98B6D961
:100DD0003ADB010B04E0B2D9010EEF6E1200AED97E
:100DE000EF6A12000901A26B01018A51220DF3CFB3
:100DF000A0F9F4CFA1F9000E0901A0270A0EA12342
:100E0000A8DAEECF98F9EECF99F9EECF9AF9EFCFB5
:100E10009BF9A6DAEECF9CF9EECF9DF9EECF9EF9C5
:100E2000EFCF9FF96DD9040E58D948DA01018F51DF
:100E3000090190270101905109019123000E92238D
:100E4000932308DBC4DADFDAE5DA01083AE197EC4C
:100E50000DF001014B2B000E4C234D234E2380DA65
:100E600012DA0901902B91239223932303DBF2DA08
:100E700077DA59DA69DA020B14E00A0EE66EE66AEE
:100E80008BC1E6FF8CC1E6FF2CD949D9125038D965
:100E900069D927D936DA0901120EA26F22D9020EBA
:100EA000DCD0040EA26F90C994F991C995F992C94A
:100EB00096F993C997F924D910D900DA12D99FDA93
:100EC000D9D042DA040B04E097EC0DF088EF09F07A
:100ED00017D9080E02D99451EE1801E0C9D09551E6
:100EE000EE1801E0C5D09651EE1801E0C1D097513F
:100EF000EE1801E0BDD001E0BBD08CDA02080AE1B7
:100F0000C2DA01E1B5D0B6DA62DA040EEF6EA0D92A
:100F10002CE3AED07FDA03082AE116DA020B01E1F6
:100F2000A7D0902B000E912392239323A3DAABDA60
:100F300006E0100EA26FD5D8040EEF6E13D0120E7D
:100F4000A26FCFD8020EEF6E942B000E952396233E
:100F5000972306DA94C9EEFF95C9EEFF96C9EEFF16
:100F600097C9EEFF75D901E383D061DA83D0C8D881
:100F7000040EB3D8EECF10F0EECF11F0B2D9E9D90C
:100F80001050EE1808E11150EE1805E11250EE185D
:100F900002E11350EE1802E097EF0DF06BDA3ADA47
:100FA000040842E170DA09E09CD8C7D906E099D874
:100FB00049D997D814DA7FDAEF82C6D9010B15E048
:100FC0000901110EA26FCCD9EFCF94F9EE2AEFCF21
:100FD00095F9EE22EFCF96F9EE22EFCF97F9EF22B7
:100FE000B8D912D97ED80A0EEF6E32D941E279D83B
:100FF00059DA05E11CDA0901100EA26F3BD0090194
:10100000A26BAED99CC9EEFF9DC9EEFF9EC9EEFF53
:101010009FC9EEFF9ED998C9EEFF99C9EEFF9AC904
:10102000EEFF9BC9EEFF24D0F5D90A0805E197EC45
:101030000DF029DA1FE01AD0EDD9050810E197EC80
:101040000DF082D9010B16E00901100EA26F81D9B3
:10105000DBD819DA0BE145D8060EEF6E0BD0DAD9E2
:10106000060808E197EC0DF00EDA04E051D902D041
:1010700097EC0DF00901A25100081EE2BAD8A2C9EE
:101080007EF190C97AF191C97BF192C97CF193C943
:101090007DF194C976F195C977F196C978F197C930
:1010A00079F12ED8DCD82CD8020E17D8DDD88BC118
:1010B00070F18CC171F1CFDC120001019151220D50
:1010C000F3CF10F0F4CF11F0000E10260A0E11220B
:1010D00010C0F3FF11C0F4FF1200E926000EEA224F
:1010E0001200A0C9E9FFA1C9EAFF120086C1E9FF09
:1010F00087C1EAFF12006DC9E9FF6EC9EAFF12005D
:101100008DC1E9FF8EC1EAFF12006DC9E9FF6EC90A
:10111000EAFF120083C9E9FF84C9EAFF1200EE5218
:10112000E9CF10F0EACF11F0E9CFE6FFEACFE6FF12
:10113000BAEC31F0126E060EE15E120088C1E9FFD2
:1011400089C1EAFF120000C9E9FF01C9EAFF1200E4
:10115000220DF3CFE9FFF4CFEAFF000EE9260A0ED5
:10116000EA221200EECF10F0EFCF11F012006CC99E
:10117000E9FF6DC9EAFF1200EECF7AF1EECF7BF105
:10118000EECF7CF1EFCF7DF1120090C9EEFF91C957
:10119000EEFF92C9EEFF93C9EEFF120001C9E9FF0D
:1011A00002C9EAFF120081C9E9FF82C9EAFF120001
:1011B000EE52E9CF70F1EACF71F12BEF05F001C9E2
:1011C000E9FF02C9EAFF120081C9E9FF82C9EAFF0B
:1011D0001200EECF76F1EECF77F1EECF78F1EFCFD0
:1011E00079F112001D0E64C3EBFF1E0E65C3EBFF09
:1011F00012000101806B816B01017F69120002C93D
:10120000E9FF03C9EAFF1200EF2AEECF90F9EF22BF
:10121000EECF91F9EF22EECF92F9EF22EFCF93F9D3
:10122000120002016C6F6D6B7FC16BF250EF0FF01B
:1012300020C9E9FF21C9EAFF12000201696F6A6B48
:101240003DEF0FF00F0EEB5002015A6F8FEF0DF0D4
:101250000101000ED8808F55000E90551200EECF80
:1012600074F1EDCF75F11200EECF72F1EDCF73F1A5
:101270001200220DF3CF00F9F4CF01F9000E002780
:101280000A0E012312004BC1EEFF4CC1EEFF4DC10F
:10129000EEFF4EC1EEFF1200100EEB6A110EEB6A6C
:1012A000280E02016C6F6D6B12007851F00BE84252
:1012B000E842E842E842040DF3501200EECF90F904
:1012C000EECF91F9EECF92F9EFCF93F91200EE6ADB
:1012D000EE6AEE6AEE6A1200CA0E105C030E115836
:1012E0001200EECF12F0EFCF13F0120082C1E9FF2F
:1012F00083C1EAFF12000F0EEB5002016B6F50EF3B
:101300000FF00D0E10C0EBFF0E0E11C0EBFF120020
:10131000A0C988F1A1C989F1CCEF06F0700EEE6E7C
:10132000170EED6E1200EE2AEE22EE22EE221200D1
:101330006CC1E9FF6DC1EAFF12000F0EEB50FF0810
:101340001200210E6DEF08F0DBDE0D0EC6DEEF5051
:101350001200C7DE180E6DEF08F0BFDE3DEF0AF099
:10136000C0DE37EF0AF0B9DEEECFDAF2EECFDBF215
:10137000EECFDCF2EFCFDDF290EC25F004C010F000
:1013800005C011F006C012F007C013F076EF08F0A8
:10139000A4DEB2EF08F0010EA0DE07C9EFFF76EF82
:1013A00008F09BDEE552E750EF6E76EF08F095DE31
:1013B000EFCF07F976EF08F090DE04C0EEFF11C022
:1013C000EEFF12C0EEFF13C0EEFF76EF08F089DEED
:1013D0001C0E83DEEF6A85DE05DF71EF08F00F0E6D
:1013E0007CDEEF681200180E78DEBCEF08F00D0E00
:1013F00074DE2FEF09F00B0E70DE34EF09F0EE52C1
:101400004ED867EF09F01F0E68DE8EEF09F07DDE23
:1014100037EF0AF066DEEF501200A9DE100E5DDE37
:1014200001015E51120067DE1C0EEB50120043D822
:10143000EF8657DE120E8FC1EBFF130E90C1EBFF4C
:101440003AD8EF8412007DDFEF501200100EA0DFBB
:101450006CEF09F085DFEECF94F9EECF95F9EECF82
:1014600096F9EFCF97F91200AADEA1EF09F0140E5A
:101470006DEF08F06EDFC5EF08F0010E2EDEEF50C5
:10148000E66E76EF08F060DF100B120087DEA1EF4A
:1014900009F023DECBEF09F0120E6DEF08F0060E17
:1014A0006DEF08F0D0DF080B120034DEA1EF09F079
:0C14B00045DEA1EF09F015DEA1EF09F008
:0414BC00966A86881E
:1014C000988802014A6B4B6B4C6B4D6B4E6B4F6BAC
:1014D0000901006B0051106E116AD890115004E69A
:1014E000010E105C000E115816E20051040DF3CFEE
:1014F00010F0F4CF11F0400E1026000E1122005112
:1015000066EC0FF010C0EFFF005166EC0FF0EE52EA
:10151000EF80002BDFD71B6A02014969F0EC0EF067
:101520007BEC0FF002011F0E78EC0FF00201656FEB
:1015300002011F0E75EC0FF07BEC0FF00201210E83
:1015400070EC0FF07BEC0FF00201080E656F0201EA
:101550000E0E8AEC0FF00A0E8AEC0FF00B0E8DECDB
:101560000FF0040E656F02010C0E8DEC0FF0020EF1
:10157000656F02010D0E75EC0FF0A2EC0FF075EC2B
:101580000FF085EC0FF0010E8DEC0FF0600E656F23
:101590000201020E75EC0FF085EC0FF0030E8DECDE
:1015A0000FF065690201070E8AEC0FF00F0E8DEC4B
:1015B0000FF0610E70EC0FF0BCC265F20201010E7B
:1015C00075EC0FF0BDC265F20201020E75EC0FF072
:1015D000BEC265F20201030E75EC0FF0BFC265F2E8
:1015E0000201040E75EC0FF0C0C265F20201050E97
:1015F00075EC0FF0C1C265F20201060E75EC0FF03A
:101600000901006B080E005D0BE202016569080E1E
:1016100009010025020175EC0FF00901002BF2D73A
:1016200085EC0FF0070E75EC0FF0440E186E0201FA
:10163000220E70EC0FF081EC0FF00D0E8DEC0FF020
:10164000E00E70EC0FF00201C00E656F0201010E9A
:101650008AEC0FF0040E8AEC0FF0010E8DEC0FF007
:10166000200E70EF0FF002010D0E95EC0FF002014D
:101670004A2711504B2302010E0E95EC0FF0020188
:101680004C2711504D2302010F0E95EC0FF0020173
:101690004E2711504F231200020149511B5C0AE1F1
:1016A0000201666BBCDB040B04E102014969A8EF8F
:1016B0000FF0000CA8EF0FF0956A6A0E8D6E010E08
:1016C000836E8D9C00000000000000000000000000
:1016D0008D8C6B0E8D6E836A8D9C00000000000067
:1016E0000000000000008D8C600E8D6E120E836E67
:1016F0008D9C0000000000000000000000008D8CA8
:10170000670E8D6E400E836E8D9C00000000000001
:101710000000000000008D8C700E8D6E50C283FFA3
:101720008D9C0000000000000000000000008D8C77
:10173000192A000E1A22120002015351541101E11C
:1017400022D1010E02015315106E116A020102012D
:101750005351102409013E6F02010201545111201E
:1017600009013F6F956A670E8D6E400E836E8D9CEA
:101770000000000000000000000000008D8C6A0ED8
:101780008D6E3EC983FF8D9C0000000000000000AC
:10179000000000008D8C6B0E8D6E3FC983FF8D9C09
:1017A0000000000000000000000000008D8C600EB2
:1017B0008D6E120E836E8D9C0000000000000000F4
:1017C000000000008D8C0201535119260201545172
:1017D0001A22700E8D6E020151C2E9FF52C2EAFF59
:1017E000512B000E5223EF50836E8D9C00000000A1
:1017F00000000000000000008D8C53C23CF954C270
:101800003DF90901010E3C5F000E3D5B09013CC939
:1018100010F03DC911F03C07000E3D5B1050111057
:1018200001E1B1D00901080E3C5D000E3D5901E215
:1018300097D0020151C2E9FF52C2EAFF512B000EBC
:101840005223EF50836E8D9C0000000000000000CA
:10185000000000008D8C020151C2E9FF52C2EAFF74
:10186000512B000E5223EF50836E8D9C0000000020
:1018700000000000000000008D8C020151C2E9FF51
:1018800052C2EAFF512B000E5223EF50836E8D9C03
:101890000000000000000000000000008D8C02012C
:1018A00051C2E9FF52C2EAFF512B000E5223EF5002
:1018B000836E8D9C0000000000000000000000000E
:1018C0008D8C020151C2E9FF52C2EAFF512B000E7A
:1018D0005223EF50836E8D9C00000000000000003A
:1018E000000000008D8C020151C2E9FF52C2EAFFE4
:1018F000512B000E5223EF50836E8D9C0000000090
:1019000000000000000000008D8C020151C2E9FFC0
:1019100052C2EAFF512B000E5223EF50836E8D9C72
:101920000000000000000000000000008D8C02019B
:1019300051C2E9FF52C2EAFF512B000E5223EF5071
:10194000836E8D9C0000000000000000000000007D
:101950008D8C080E09013C5F000E09013D5B62D7CA
:10196000020151C2E9FF52C2EAFF512B000E52237D
:10197000EF50836E8D9C000000000000000000000E
:1019800000008D8C43D71200956A6A0E8D6E010E91
:10199000836E8D9C0000000000000000000000002D
:1019A0008D8C6B0E8D6E836A8D9C00000000000094
:1019B0000000000000008D8CFF0E195C28E15F0E16
:1019C0001A5C25E109013269336932C967F233C90A
:1019D00068F238DA600E8D6E0A0E836E8D9C000000
:1019E000000000000000000000008D8C0201100EBD
:1019F000666F15DA0901316F0901326B0901440E76
:101A0000336F32C967F233C968F21CDA1CD0600E3A
:101A10008D6E0A0E836E8D9C000000000000000099
:101A2000000000008D8C9568700E8D6E8D9A000000
:101A30000000000000000000000083CF31F98D8A13
:101A4000192A000E1A220901315100D0120057C282
:101A5000B5F958C2B6F902015751581103E1F36ABA
:101A6000F46A56D0956A6A0E8D6EB5C983FF8D9C57
:101A70000000000000000000000000008D8C6B0ED4
:101A80008D6EB6C983FF8D9C000000000000000031
:101A9000000000008D8C600E8D6E0A0E836E8D9C92
:101AA0000000000000000000000000008D8C090113
:101AB000B55119260901B6511A22600E1A5C02E3CB
:101AC0001C0E1A5E9568700E8D6E0901B5C910F076
:101AD000B6C911F0B507000EB65B1050111013E037
:101AE0008D9A0000000000000000000000000201CC
:101AF00055C2E9FF56C2EAFF552B000E562383CF8D
:101B0000EFFF8D8AE2D757C2F3FF58C2F4FF00D02F
:101B1000120002015951DAD9EE52EF90120002017F
:101B20005A51D4D9EE52EF805AC21BF0120018C09D
:101B300036F90901010E356FE8CF67F218C068F277
:101B400081D922DF0901346FE8CF65F20201030E6B
:101B500075EF0FF0E5D90901006F0201200EC0D921
:101B600018500901005D05E2600ED8801854002568
:101B700002D01850005D016FE850106E116A1C0E03
:101B8000D8801056000E115610C001F910C003F98C
:101B9000026B02C9F3FF10C0F4FF12000201E00E55
:101BA000CCD90901006F0201200E9AD90901005118
:101BB000040B01E0000C010C5DC2E9FF5EC2EAFF0C
:101BC000EF68AED90901126F0201200EB6D90901E2
:101BD000136FC3D9100B37E00201666B20D9040BD9
:101BE0000901176F0201210E7BD9020EE66E97ECF8
:101BF00035F0E55286D90A0E8DD90B0E76D909013A
:101C0000175108E0AAD90A0B02E0000E01D0010E1C
:101C10000901176F0201020E656F02010D0E7DD9D9
:101C2000220E5ED912C918F082DF02016569020135
:101C3000070E70D90D0E59D90901175103E00201A1
:101C4000260E4ED9000C09011351125D67E013C92D
:101C500015F9146B14C967F213C968F2F3D8120EA0
:101C60000201576F586B0201000E556F090E566F37
:101C7000EEDE09010051010B4EE0400E025D000E48
:101C8000035949E3EE0ED8800255050E035543E390
:101C9000600E015D40E20151106E116AD890115042
:101CA00004E6440E105C000E115835E310C9D8F25A
:101CB00011C9D9F28BEC25F0F3CF10F9F4CF11F95B
:101CC000060EE66EE66A0A0EE66E090EE66E5BC268
:101CD000E9FF5CC2EAFF5BC210F05CC211F05BC2BC
:101CE000E6FF5CC2E6FFBAEC31F0126E060EE15E72
:101CF0001250080E0901115D0BE1105103E0060EB0
:101D0000105D06E15DC2E9FF5EC2EAFF10C9EFFFA8
:101D100013C918F0010C12C918F009DF000C0201F8
:101D20000A0E656F0201070EE0D804D9EFCF41F922
:101D30000901406B40C967F241C968F283D8060EB9
:101D40000201536F546B5FC251F260C252F2F4DC75
:101D5000BCC250F2B1DCBDC250F2AEDCBEC250F229
:101D6000ABDCBFC250F2A8DCC0C250F2A5DCC1C2DD
:101D700050F2A2DC0201615103E10901426B03D080
:101D80000901060E426F0201080E506F95DC42C930
:101D900050F292DC0E0E02016227000E63233C0E0D
:101DA000625D000E635903E23C0E626F636B62C2B8
:101DB00040F963C241F962C265F20201050E95D88D
:101DC00041C965F20201060E75EF0FF0BBD8A5D828
:101DD000240E86D81BC049F2ADD8EE52EF80120017
:101DE0009568600E8D6E8D8C8D8A8D8E966A0A0E2A
:101DF000E66EEFEC35F0E5527ED88D9E1200600E57
:101E0000020164118D6E65C283FF956A8D9C00008E
:101E1000000000000000000000008D8C120095689A
:101E2000600E020166118D6E8D9A000000000000A8
:101E300000000000000083CF37F98D8A0901375177
:101E400000D0120067C219F068C21AF067C265F2CA
:101E50000201080E4AD868C265F20201090E75EF48
:101E60000FF00201090E44D80901016F0201080EAA
:101E70003FD8F36E01C9F4FF120018C023F909011D
:101E8000120E226F020169510901222702016A51D3
:101E90000901232322C967F223C968F222EF0FF058
:101EA0006BC21BF047D8EFCF0DF909010E0E0C6F76
:101EB00002016C5109010C2702016D5109010D232A
:101EC0000CC967F20DC968F222EF0FF0E96EEA6AF9
:101ED000D890E936EA36460EE926020EEA221200CA
:101EE000656F0201646BFFEF0EF0646FFFEF0EF0A1
:101EF000666F0FEF0FF0050EE66E97EC35F0E552CA
:101F000012000201656B020112000201440E656FAE
:101F100002011200EADF81EF0FF0E7DF0201120099
:101F20000201600EDDDFADEF0FF0E2DF106E116A2F
:101F3000E85012001B5066EF0FF0D2DF0201030ED3
:101F400078EF0FF0F7DFEFCF65F20201040E120019
:101F5000F1DFEE52EF50010B12000201070E78EF95
:021F60000FF080
:0E1F62000B01AA6B64C3A4FB65C3A5FB0901B8
:101F7000036B080E035D15E2500E01014F6F506BAD
:101F80006EEC00F0E66E0901E3DBF9EC13F0E0DB48
:101F9000020EC0DBEF6ADCDB090EBCDBEF6A032B51
:101FA000E8D71200ABCB00F9ACCB01F9090100C9AD
:101FB000E9FF01C9EAFF002B000E0123EF502E08B4
:101FC00007E000C9E9FF01C9EAFFEF50EFE10A0CA1
:101FD000026B0251106E116A100E105C000E115847
:101FE00014E20251A0DB00C9E6FF01C9E6FF08ECDC
:101FF00032F0136E050EE15E1350000903E1090192
:10200000025112000901022BE4D70A0CBFDB04E0E5
:10201000200E0901005DFAE00901016B2B0E090198
:10202000005D02E1200E006F2F0E005D1FE05C0ED0
:10203000005D1CE0200E005D1BE03F0E005D18E01F
:102040000D0E005D15E00A0E005D12E00C0E015D44
:102050000DE2610E005D05E300517A0802E3200EF7
:10206000005F0151012BAADB00C9EFFF8FDBD6E136
:1020700009010151A3DBEF6A090101510CE1030ED3
:10208000106E6A0E93DBAECBE6FFAFCBE6FF1EEC25
:1020900032F0050EE15E3F0E0901005D01E1010C29
:1020A000000C0B01A4510301645D106E65510B011E
:1020B000A555116EE00E105C2E0E115801E3AA6BAF
:1020C0000901876B080E875D06E287C9B0FB04D85B
:1020D0000901872BF7D712000B01B0510A0DF3CF7E
:1020E0007CF9F4CF7DF9540E09017C270B0E7D237A
:1020F000010E7A6F09017A5101E182D17A6B05DB19
:1021000064DB0AE17CDBEF50020B01E0AFDB77DB45
:10211000EF9479DBEF6A1200F8DA020EEB50070A4F
:10212000E9E0010A01E15CD1030A01E12DD1010AD4
:10213000E1E0070ADFE0010A01E118D1030A01E149
:10214000D6D0010AD7E1E1DA4DDBD4E00901010E76
:102150007A6F64C3A4FB65C3A5FB51DBEF6A6ADB3E
:102160000B01B66FAAD90901796F49DBEF9462DBE5
:102170000101916F5DEC08F067DBEE52060ECADAE2
:102180000B01A651EE1820E1A751EE181DE1A85150
:10219000EE181AE1A951EE1817E116E1AA5102E072
:1021A0002EDBEF84020EAA5D02E0000E01D0010ECC
:1021B000106E25DB1050010BF36EF346F346F34629
:1021C000F70EEF14F310EF6E0901795101E089D099
:1021D0000B016C0EAE6F090EAF6F2CDB0B01AD6FF8
:1021E00015DF0901806F580E6C5D15E108DBEF50BB
:1021F000040B11E10A0EE66EE66A0D0E106E6A0E11
:10220000D5DA6C0EE66E090EE66EE5EC31F0136E73
:10221000070EE15E13500B016C0EAB6F090EAC6F35
:10222000C1DEE66EEADAE5DA090180510BE0010170
:102230006C0EE96F090EEA6F7CC9E7F17DC9E8F120
:10224000F6EC15F018DBDFDA050EEF6EE6DAD1DA20
:1022500000DB106E060E105C30E312DB04082DE389
:102260006C0EE66E090EE66E37EC32F0E552E55282
:10227000F3CF7BF905DB030802E3030E01D0020E66
:1022800009017B5FFDDA0B0FE66EB7DAB2DAF8DA36
:102290004ADA7B51146A6C0F136E090E142213C0B4
:1022A000E6FF14C0E6FF1EEC32F0156E050EE15E8F
:1022B0001550B3DAE552E750EF6ECBDAFF0803E1D1
:1022C000D3DAEF6A06D0C5DAFE0806E1CDDA030EEE
:1022D000EF6E99DA050E82D092DAEF8294DA010E6F
:1022E0007DD0790501E006D78EDA030E77D0B5DA16
:1022F00001E100D70901010E7A6F0B018C0EBB6F53
:10230000690EBC6F4EDA0B019C0EBB6F690EBC6F81
:10231000A7DA73DAEF34EA6AFE0BEA36E96E6E0E7C
:10232000E926020EEA22EECFBBFBEDCFBCFB39DA89
:1023300064DAEFCF10F00B0E105C06E30B01AB0E6E
:10234000BB6F690EBC6F8CDAB0CBB9FBA6D998DA3B
:10235000060803E154DAEF8002D051DAEF90D5D9C4
:10236000030ED8D9EF6A4FDA020E38D0CED93ADA56
:1023700001E081DA7CC9B7FB7DC9B8FBDCD8000974
:1023800001E1B8D673DA28D068DA01E1B3D66CDAA5
:10239000EF34EA6AFE0BEA36E96E8E0EE926020E8B
:1023A000EA22EECF7EF9EDCF7FF909017EC9F6FF73
:1023B0007FC9F7FF7E2B000E7F230800F5CF7BF946
:1023C000F55005E07BC95AF1A0D9D1D9EED732DA60
:1023D0000101576F75EC01F016DA060EEF6E8AD622
:1023E00094D9F3D90AE039DA08E024DA0101566F0A
:1023F00035EC01F008DA070EEF6E01DAEF947AD6C9
:102400001200B4CBE9FFB5CBEAFFEF0409011E6F60
:102410001D6BEF6A1F6B1E510B01EA6AB225E96E54
:10242000B351EA22EF6A09011F5141E101011C0E7B
:10243000626F090E636FB1CB61F1B9EC02F0000974
:1024400036E03D0E09011C5D0BE11C6B1E511D5D4C
:102450001EE21D29B4CBE9FFB5CBEAFFEF6E17D022
:10246000260E1C5D02E1020E0AD0200E1C5D06E065
:102470000D0E1C5D03E00A0E1C5D04E1010E1F6FD2
:102480001C6B05D02B0E1C5D02E1200E1C6F1E5133
:102490001D5D06E2B2CBE9FFB3CBEAFF1CC9EFFF3B
:1024A0000B01B22B000EB32309011D2BBCD7090170
:1024B0001F5101E1000C1F0512000901056B040EFC
:1024C000055D19E205510101626F636B000E622721
:1024D000090E6323B6CB61F1B9EC02F000090BE001
:1024E00009010551052BEA6A000FE96E090EEA227F
:1024F000EF502008E4E109010551EA6A000FE96E96
:10250000090EEA22EF6A470E005D07E1450E015D04
:1025100004E1540E025D01E1000C500E005D0AE181
:102520004F0E015D07E1530E025D04E1540E035DA1
:1025300001E1010C020CF2D813D901E1A6D0090186
:10254000856BECD8030EEB50040818E0E7D814D9DB
:10255000400B0DE1E3D8010EEB500201386FA6EC01
:1025600024F00901866FDAD807D9200B07E0D6D806
:10257000EF500101576F75EC01F0010CCFD8090E37
:10258000C9D8EF50010B01E17BD0C8D8030EEB5046
:10259000040A50E0070A34E0010A1BE0030A0BE0DA
:1025A000010A6BE1250E865D03E131D9010E26D0CB
:1025B000010E856F62D0250E865D03E1010E856FE9
:1025C0005AD029D9030EA6D886C9EFFF20D9020E0A
:1025D00015D0610E865D02E3270E04D0410E865DA4
:1025E00002E3070E865F300E865D100DF350E66E37
:1025F00012D9020E8FD8FDD80AD9030EEF6E3DD046
:10260000610E865D02E3270E04D0410E865D02E373
:10261000070E865F300E865D106EFDD8020E7AD8EA
:102620001050EF12F4D8040EEF6E78D873D8EE6A1B
:10263000ED6A23D00101860EED6F090EEE6FB7CB68
:10264000EBF1B8CBECF193EC16F0F3CF10F0F4CF44
:1026500011F0E1D8F3CFEEFF11C0EDFF0901010E3B
:10266000856FD9D8FF0EEE1808E1FF0EED1805E1D1
:10267000865101E1856BCBD8EF6A855101E15BD7CB
:1026800086C95AF14BD873D856D748D8010EEB50AB
:102690000201376F7FEC24F0000C0B01B9510A0DD9
:1026A000F3CF85F9F4CF86F9540E090185270B0E77
:1026B000862301010D0EC1D801010A0E1DEF14F091
:1026C0000B01BA510A0DF3CF85F9F4CF86F9540EF8
:1026D000090185270B0E8623BBCBF6FFBCCBF7FF8A
:1026E0000800F55011E00B01BBCBF6FFBCCBF7FFA8
:1026F000BB2B000EBC230800F5CF5AF185C9E9FFBA
:1027000086C9EAFF34D8E8D712007CC9E9FF7DC941
:10271000EAFF1200E926000EEA221200B7CBE9FF19
:10272000B8CBEAFF1200040DF3CFF6FFF4CFF7FFAA
:102730004C0EF626690EF722F6CF10F0F7CF11F007
:10274000126A10C0E6FF11C0E6FF12C0E6FF1200D9
:1027500003510A0D79D8540EE9260B0EEA22120015
:10276000EF500101586FD9EC01F000091200EF5051
:102770000101596FF2EF01F0010EEB50080D64D822
:10278000000EE926020EEA22EF5012000101000EAF
:10279000626F090E636FADCB61F1B9EC02F0000915
:1027A00012005ED8B0CBB9FB4DEF13F0116E126A78
:1027B00010C0E6FFE66E12C0E6FF12000B01EA6AE7
:1027C000AE25E96EAF51EA221200EF500101556FBC
:1027D0002CEC01F000091200010EEB500201366FE3
:1027E00077EF24F0EF500101696F44EC03F000092A
:1027F0001200E552E750EF6E120036D844D085DF64
:10280000090E8AEF13F081DF020E8AEF13F086DFE4
:10281000030E8AEF13F082DF36D00201356B02011E
:102820006C0E336F090E346FDAEC23F0E66E6DDF59
:10283000EE5212006ADFEF5012005A6F85C9E9FFAD
:1028400086C9EAFFB7EF13F0F3CFE9FFF4CFEAFF51
:1028500012005BDF010EEB50120057DFB0EF13F0F8
:10286000B0CBBAFB60EF13F050DF0DD0C8DFEF92B2
:102870004CDFECEF13F0DEDF0101606F9BEF02F045
:0C288000BCDFEF501200040E8AEF13F0D2
:04288C001200A6ECA4
:1028900018F0040B06E0A6EC18F0080B01E0020C9F
:1028A000010C000C09011C6B1D6BE2C1E9FFE3C1C7
:1028B000EAFFEF506B0801E080D00901010E206FA4
:1028C0000201210EE76F090EE86F010E0101E225FA
:1028D0000201E56F000E0101E3210201E66F95ECB4
:1028E00026F0000903E1F36AF46A7FD1E4C1E6FF50
:1028F000E5C1E6FF75EC2CF0E552E552F3CF22F985
:1029000009012151110804E2160E0901215D05E1BA
:1029100009011C830901206B43D0090121511508CD
:1029200009E3130E0901215D04E009011C8F09016F
:10293000206B36D0090121511A0801E331D0090179
:1029400021511E0801E32CD009012151220817E36F
:102950001F0E0901215D04E0210E0901215D07E13F
:1029600009012251080802E30901206B02D0090184
:10297000206B0901205102E109011C8511D00901D8
:102980002151300805E309011C870901206B08D09B
:1029900009012151320804E309011C890901206B56
:1029A0000901205109E10101E65106E022C9A8FF11
:1029B00021C9D7F2B0EC32F013D1E2C1E9FFE3C193
:1029C000EAFFEFCF10F0610E105C01E2B5D0E2C17A
:1029D000E9FFE3C1EAFFEF50670801E2ADD0E2C1D1
:1029E000E9FFE3C1EAFFEF50640807E0E2C1E9FF55
:1029F000E3C1EAFFEF50650803E1F36AF46AF5D03A
:102A0000E2C1E9FFE3C1EAFFEF509F0F09011E6F2A
:102A10001F6B890E09011E270F0E09011F23010ECE
:102A20000101EA6AE225E96EE351EA22EF5014E17E
:102A30000201200EE76F090EE86FE4C1E5F2E5C17F
:102A4000E6F295EC26F0000906E01EC9E9FF1FC971
:102A5000EAFF20C9EFFF6FD0010E0101EA6AE2250B
:102A6000E96EE351EA22EF50780833E1020E0101EA
:102A7000EA6AE225E96EE351EA22EF50D00F106EC8
:102A8000010E105204E0E846FE0B1006FCE10901BD
:102A9000206FE4C1E9FFE5C1EAFFEF5031080AE128
:102AA0000901201D106E1EC9E9FF1FC9EAFF105061
:102AB000EF160ED0E4C1E9FFE5C1EAFFEF503008A0
:102AC00007E11EC9E9FF1FC9EAFF09012051EF1202
:102AD00032D0010E0101EA6AE225E96EE351EA22F1
:102AE000EF50D00F106E010E105204E0E846FE0BBE
:102AF0001006FCE10901206FE4C1E9FFE5C1EAFF2E
:102B0000EF5030080AE10901201D106E1EC9E9FFCF
:102B10001FC9EAFF1050EF160ED0E4C1E9FFE5C16E
:102B2000EAFFEF50310807E11EC9E9FF1FC9EAFFBC
:102B300009012051EF1254D0E2C1E9FFE3C1EAFFDD
:102B4000EF506C082DE10101E65129E0010E010171
:102B5000EA6AE225E96EE351EA22EF50610A11E0E8
:102B6000030A01E01CD00201080EED6FE4C1EBF294
:102B7000E5C1ECF23E0E0201E96FEA6BBAEC26F019
:102B80000ED00201080EED6FE4C1EBF2E5C1ECF2EC
:102B9000350E0201E96FEA6BBAEC26F000D020D0C6
:102BA000E2C1E9FFE3C1EAFFEF506D0819E101015D
:102BB000E65116E0E4C1E9FFE5C1EAFFEF50720A11
:102BC00001E00ED0F0EC0EF0FF0E986E966E956E52
:102BD000936E000E866E846E836E816EFF0000D051
:102BE0001CC9F3FF1DC9F4FF00D012000901146BCA
:102BF000156B186BE7C1E0F1E8C1E1F148DE0901AE
:102C0000196F140E166F0B01160EB46F090EB56F07
:102C10000B01000EB26F090EB36FB1DAEF500B016A
:102C2000B16F01EC12F00901176F182B1B6B6C0EC2
:102C3000005D36E10151750A2BE0050A45E1010E00
:102C40001B6F3E0E54DA40E1020E0901185D3CE1B3
:102C5000010E1A1539E093DAEF500101916F5DEC26
:102C600008F0F3CFE9FFF4CFEAFFEE52060E83DA65
:102C7000EECFA6FBEECFA7FBEECFA8FBEFCFA9FBD5
:102C80000B01010EAA6F43DAEF8441DAEF961CD0F4
:102C9000010E1B6F350E2BDA17E109011A8114D0D2
:102CA0006D0E005D11E119510FE01651EA6A000F37
:102CB000E96E090EEA22EF506F0A06E1010E1B6F62
:102CC0000B01AA6B24DAEF9409011B5115E119C914
:102CD000E6F116510101E46FE56B000EE427090EE1
:102CE000E5230101000EE26F090EE36FDBDDF35017
:102CF00009011413F4501513175101E082D7145130
:102D0000020B01E012001451040B02E0C4EF32F098
:102D10001451080B02E013EF33F01451100B02E0D2
:102D20003FEC33F01200F7D9020E25DAEFCF01F9AC
:102D3000F2D9030E20DAEFCF02F9EDD9EECF07F981
:102D4000EDCF08F913DAEF6AEBC1E0F1ECC1E1F184
:102D50009EDD0901096F610E025D6DE30251680895
:102D60006AE3006B610E025D066F070E0115106EBF
:102D7000010E105204E0E846FE0B1006FCE10901CA
:102D8000056F0651036F046B920E03270F0E042389
:102D9000D0D909E10651036F046B890E03270F0E8A
:102DA0000423008107D00651036F046B800E0327B4
:102DB0000F0E0423F00E0115066FE85004E1B9D997
:102DC00034E0310E35D0100E065D0CE1B2D905E1CC
:102DD0000101EC0EF26F6A0E02D10101E90EF26FF1
:102DE0006A0EFDD0200E065D03E1010E001506E01F
:102DF000300E065D08E1010E001505E0080E011514
:102E000001E1D8D0E8D0400E065D08E1010E0015C2
:102E100005E00101CF0EF26F6A0EE1D0500E065DA3
:102E200001E0E6D0010E001502E0300E01D0310EB7
:102E30009DD9EF6EDDD06B0E025D0AE1095101E113
:102E4000D7D001C9D6F2A6EC32F00101FC6F62D0F6
:102E50006C0E025D42E109512CE00151040A24E0AC
:102E6000060A1DE0030A16E0010A01E0C1D00905C7
:102E70000CE1350E0101F76FF86BEDC1F5F1EEC114
:102E8000F6F107C9F4F11AEF18F00101530EF26FD1
:102E9000520EA5D00101F40EF26F6B0EA0D001010D
:102EA000FA0EF26F6B0E9BD00101500EF26F520EB4
:102EB00096D00151030A08E0030A01E099D001010C
:102EC0004A0EF26F520E8BD0095102E1300E01D042
:102ED000310E066FE8CFFCF11DD06E0E025D01E0F1
:102EE00087D0006B0F0E0115106EC11C0F0B105C0C
:102EF00001E20083F00E0115066FE85005E10101C3
:102F0000B60EF26F6A0E6BD0100E065D0BE126D97D
:102F1000EFCFFCF1EDC1FAF1EEC1FBF107C9F9F118
:102F20003BEF18F0200E065D39E118D9EFCF06F916
:102F30000751081120E1330E03D90750300F01016A
:102F4000DA6F2E0EDB6F330EFBD803C006F90901D2
:102F500003500A0DB8D80101DC6F0A0EF1D807C082
:102F600006F909010750640DAED80101DD6FDE6B73
:102F70000901076B086B0751D5D8F8D8EF6E0751D8
:102F8000D1D836E007C910F008C911F0072B000EA0
:102F9000082307C9F3FF08C9F4FF1200300E065DCD
:102FA00003E1020E001506E1500E065D08E1020E77
:102FB000001505E10101E00EF26F6A0E10D0400E1F
:102FC000065D03E1020E001506E1600E065D10E1EC
:102FD000020E00150DE10101E50EF26F6A0EF36FAE
:102FE000EDC1F0F1EEC1F1F107C9EFF1FBEF17F020
:102FF000F368F46812000101EF51F76AF225F66EEA
:10300000F351F7220800F550F0C1E9FFF1C1EAFFE2
:10301000EF6EF0C1E9FFF1C1EAFFEF5003E1F368A1
:10302000F4681200EF2BEF51116AEFC1F3FF11C0EA
:10303000F4FF12000101F451F72509010A6F000E97
:103040000101F821AA6E0AC9A9FF3F0EA616A680A3
:10305000A850F5C1E9FFF6C1EAFFEF6EA85003E101
:10306000F368F4681200F42BF451116AF4C1F3FF11
:1030700011C0F4FF12000101F95110E1DA0EE66E01
:10308000010EE66EFC51E66EE66AEAEC2CF0E552C3
:10309000E552E552E5520101DF6BF96BF95142D877
:1030A000FAC1E9FFFBC1EAFFEF6EF9513BD803E13A
:1030B000F368F4681200F92BF951116AF9C1F3FFB2
:1030C00011C0F4FF1200F3CF10F0F4CF11F0330E63
:1030D0000B6E0C6AF3CF06F0F4CF07F0AEEC35F0D0
:1030E00006C010F007C011F0300E062412000201D5
:1030F000F06FF16B090116510201EE6FEF6B000EDC
:10310000EE27090EEF23F2EC26F00009120037D863
:10311000090EBBEF18F0EBC1E9FFECC1EAFF040EAA
:10312000BBEF18F0EA6ADA0FE96E010EEA22EF50FF
:10313000120003C9E9FF04C9EAFFEF5005151200A8
:10314000106E0C6E06C907F0D5EF35F0E0C1E9FF4F
:10315000E1C1EAFF090E0FD8EF5012000F0E011562
:10316000EA6ACA0FE96E020EEA221200EDC1E9FF17
:10317000EEC1EAFF1200E926000EEA221200E7C1C2
:08318000E9FFE8C1EAFF1200BB
:083188000901006B020E005D5D
:1031900007E200513BDB00512DDBEF90002BF6D70F
:1031A00012000901000E016F010E026F006B020E8A
:1031B000005D43E2DCDA0C0EC7DACADA126A136A7F
:1031C000105011101210131032E1D1DA0C0E29C177
:1031D000EBFF0D0E2AC1EBFF01012B512C1111E069
:1031E0000A0EE66EE66A2BC1E6FF2CC1E6FFBFDAE7
:1031F00001C910F002C911F001C9E6FF02C9E6FFDA
:10320000D8DAB5DA0A0E2DC1EBFF0B0E2EC1EBFF9B
:10321000AEDA0E0EEB6A0F0EEB6AA9DA100EEB6A4D
:10322000110EEB6A00C928F1090100511200140EB9
:103230000127000E0223002BBAD7FF0C01012F51EA
:1032400006EF1CF0020E0101305D04E230C128F1EE
:103250004CEF0BF0000C01012851140DF3CF0AF9CB
:10326000F4CF0BF9000E09010A27010E0B23CADA6D
:10327000EE50ED1004E190DA94DA8EDA87DA31C19B
:1032800050F25CEC0BF0BEDAEE2AEF22BBDAC4DAC5
:1032900001E346D8010C01012851140DF3CF0AF9BE
:1032A000F4CF0BF9000E09010A27010E0B23A6DA51
:1032B000EE50ED1004E151DA74DA4FDA67DA9EDA93
:1032C00001013451EE24106E3551EE20116ED60EF0
:1032D000D8801054030E11540AE290DAEECF34F184
:1032E000EFCF35F1D60ED8803457030E355734C1A1
:1032F00053F235C154F232C151F233C152F29CEC57
:103300000BF07CDA01013451EE263551ED2276DAEC
:1033100083DA01E305D834C1F3FF35C1F4FF1200AD
:1033200001012851140DF3CF08F9F4CF09F9000E6B
:1033300009010827010E092315DA0C0E05DA40DA17
:10334000F3CF00F9F4CF01F90DDA0A0EFDD938DA1E
:10335000F3CF02F9F4CF03F905DA0E0EF5D9EECF6B
:1033600004F9EFCF05F9080E09010427000E052323
:10337000066B076B140E02016C6F6D6BF3D906DAE6
:1033800004C957F305C958F30301110E566FEAD962
:1033900008C954F309C955F3F6EC27F004C9D8F26B
:1033A00005C9D9F28BEC25F0F3CF04F9F4CF05F978
:1033B000080E0201536F546B0201000E516F090E8B
:1033C000526F9CEC0BF0E6EC0EF0CCD9120EBCD98F
:1033D000EF68C8D90E0EEB6A0F0EEB6A1200020EF0
:1033E0000101365D0AE236C128F1FFD9D880EE54DA
:1033F000000EED5401E3000C010C000C17DA01E1A2
:10340000000C2851F7D9EF50010B01E013DAC4EC9E
:103410000CF037C1E9FF38C1EAFFEF6E11DAEE06B2
:10342000EF5AE3D9EE50ED1002E197EC0DF0010CEC
:10343000FDD903E1F36AF46A12002851DBD9EF5099
:10344000010B01E0F7D9FCD983D93B51105C3C5109
:10345000115805E2CAD9EECF3BF1EDCF3CF13BC1AB
:1034600057F23CC158F239C155F23AC156F227EC35
:103470000DF0F3CF00F9F4CF01F9E2D909010051C1
:10348000EE5E0151ED5AD2D902E197EC0DF03BC14D
:10349000F3FF3CC1F4FF1200C9D902E097EC0DF034
:1034A000CFD9EE6AED6A1200080E0201576F586B11
:1034B0000201460E556F090E566F27EC0DF046C9F6
:1034C0005DF947C946F95DC947F948C95DF949C978
:1034D00048F95DC949F9080E106E09014B51D880B1
:1034E000105403E24A055D6F02D04AC95DF9080E27
:1034F0004B5D4A6F5DC94BF94CC95DF94DC94CF93B
:103500005DC94DF93DC1E9FF3EC1EAFF060E1CD978
:10351000EECF4FF9EECF50F9EECF51F9EFCF52F990
:1035200055D9EFCF53F9010E0FD9EFCF54F94ED93A
:10353000020E0AD9EFCF55F949D9030E05D9EFCFBD
:1035400056F9576B110E586F41C159F942C15AF9DA
:1035500041C1D8F242C1D9F28BEC25F0F3CF59F931
:10356000F4CF5AF90C0E0201E06FE16B02014F0E2D
:10357000DE6F090EDF6FBFEC25F0F3CF5BF9F4CF00
:103580005CF909015B1F5C1F1A0EFBD85BC950F286
:103590005CEC0BF05CC950F25CEC0BF0140EF1D853
:1035A00041C1E2F242C1E3F21BEC26F0F3CF5BF93A
:1035B000F4CF5CF909014C51F31816E14D515C1937
:1035C00013E13FC147F140C148F13DC145F13EC162
:1035D00046F10101460E436F090E446F1CD80901E4
:1035E0004E6FFF0E4E5D03E197EC0DF0010C4E5156
:1035F000A1D8100EA9D84AC9EEFF4BC9EDFF4E5114
:10360000F9D8EF80010C0101285194D8E9CFF3FFDC
:10361000EACFF4FF120009010169000E026F010EEA
:10362000036F006B020E005D5BE2A6D80C0EFAD8A9
:10363000020E8AD8D5D80001125010184AE1135052
:10364000111847E199D80A0EEDD8CAD812501018AF
:103650003EE1135011183BE18FD8100E75D8EECF14
:1036600014F0EFCF15F0166A176A145015101610E3
:1036700017102DE145C1E9FF46C1EAFF060E64D8E7
:10368000EECF10F0EECF11F0ABD876D8060E5CD8A6
:10369000EE50101808E1EE50111805E1EE50121826
:1036A00002E1EE50131810E047C1E9FF48C1EAFFFC
:1036B000E868EE180CE1E868EE1809E1E868EE1831
:1036C00006E1E868EE1803E109010051120000C9A3
:1036D00001F90901140E0227000E0323002BA2D7C3
:1036E000FF0E015D24E00151140DF3CF02F9F4CF78
:1036F00003F9000E0227010E03230A0EE66EE66AA6
:1037000045C1E6FF46C1E6FF37D802C910F003C93C
:1037100011F002C9E6FF03C9E6FF4BD85CD818D800
:103720002BD80A0E10C0EBFF0B0E11C0EBFF0901E6
:1037300001511200140DF3CFE9FFF4CFEAFF000EA0
:10374000E926010EEA221200E926000EEA22120002
:10375000EECF10F0EFCF11F012000AC9E9FF0BC94C
:10376000EAFF120008C9E9FF09C9EAFF120001C90E
:10377000E9FF02C9EAFF120002C9E9FF03C9EAFF33
:1037800012000201696F6A6B3DEF0FF0120EEB50F1
:1037900002016B6F50EF0FF00AC9E9FF0BC9EAFF96
:1037A0001200120E1BC0EBFF1C0E02016C6F6D6B42
:1037B0001200BAEC31F0126E060EE15E12501200E9
:1037C000EECFD8F2EDCFD9F28BEF25F03FC1E9FF74
:1037D00040C1EAFF120043C1E9FF44C1EAFF120001
:1037E000EECF12F0EFCF13F012002851A3DF100E2E
:1037F000A4EF1BF09FDF130EA4EF1BF0AEDF0E0E45
:10380000A4EF1BF0C9DF0E0EA4EF1BF093DF0C0E2C
:103810009BDFEE6AED6A12009BDFD60E105C030E92
:103820001158120091DF94DFEBEF1BF009D8EE5036
:10383000ED1012002851DEDFEF901C0EC1EF1BF0DF
:063840000101F5EF1BF091
:0A384600070E0301755D01E1120099
:10385000FF0E765D01E0A7DA03017669756B786B80
:10386000120003017551060A01E1A2D0030A66E0C5
:10387000010A59E0070A46E0010A33E0030A27E09B
:10388000010A01E0120009010E690F69106911694E
:103890001269136914691569166917690301086BC0
:1038A000096B0A6B0B6B430E01012D6F2E6B01012F
:1038B0000E0E2B6F090E2C6F440E0101296F2A6B1F
:1038C000D1EC18F00301766F62DA010E756F50DAF1
:1038D000140E105C000E115801E27DD00301020E9F
:1038E0003BD00301085109110A110B1133E176C3D2
:1038F00030F122EC19F000096EE00301010E5FDAED
:10390000030E2AD061DA03E30301020E756F76C35A
:1039100036F1EFEC19F000095EE063D802085BE1D4
:103920000301040E756F76C330F122EC19F0000923
:1039300052E00301030E43DA050E0ED076C336F1D2
:10394000EFEC19F000092EE04CD80901186F060EB3
:10395000185D04E10301040E756F1200050E185D79
:1039600026E121DA0301766912DA060E756F08C3C3
:10397000B8F209C3B9F20AC3BAF20BC3BBF210C35F
:10398000C2F211C3C3F212C3C4F213C3C5F20CC313
:10399000C6F20DC3C7F20EC3C8F20FC3C9F27781D6
:1039A000782B120011DA17E30301020E756F120073
:1039B000DFD9640E105C000E11580DE30407000EF1
:1039C000055B065B075B045105110611071102E157
:1039D0000301756BDCD912000301080E756FD3EF7C
:1039E0001EF00901026B03013C0E046F056B066BB0
:1039F000076BB0D9020E0901005D01E0EBD0016B4D
:103A00000F0E015D02E2EFD9FBD70101080E376FFF
:103A1000030EABD9090E376F030EA7D90A0E376F05
:103A2000030EA3D90B0E376F030EC6D90901016B24
:103A3000080E015D02E2D7D9FBD7BCC208F9BDC2AE
:103A400009F9BEC20AF9BFC20BF9C0C20CF9C1C262
:103A50000DF9016B060E015D0EE27CD909010151E1
:103A6000EA6A080FE96E090EEA22EF50005D01E0F4
:103A7000D3D0012BEFD7016B0151106E116AD89092
:103A8000115004E6CE0E105C000E115802E2ABD9C4
:103A9000F3D7036B5FD909010051330A62E0CC0A06
:103AA0005DE0C90A47E0350A23E0020A0DE0340A66
:103AB00001E07DD04FD90901000501E0ADD0010141
:103AC000020E376F090E48D072D901E0A5D001016E
:103AD000100E376F030E49D9110E376F030E45D9FB
:103AE000120E376F030E41D9130E376F030E34D009
:103AF0005ED901E291D001010C0E376F030E35D96A
:103B00000D0E376F030E31D90E0E376F030E2DD900
:103B10000F0E376F030E50D9040E0901005F090123
:103B200000510007000952E00101010E376F090E34
:103B300043D9F5D73CD970E10101070E376F090E63
:103B400014D9060E376F090E10D9050E376F090EFE
:103B50000CD9040E376F090E2FD938D0010E036F20
:103B600035D025D959E10101070E376F030EFDD875
:103B7000060E376F030EF9D8050E376F030EF5D812
:103B8000040E376F030E18D9D880080E03010455B0
:103B9000070E0555000E0655000E075517E2080ED4
:103BA000045F070E055B000E065B075B0FD001018B
:103BB000000E376F090E00D90901005100070009F6
:103BC00005E00101010E376F090EF5D70901035118
:103BD00001E160D7020E025D09E104C900F305C9E5
:103BE00001F306C902F307C903F311D0000EE96E11
:103BF000030EEA6EEE50041908E1EE50051905E1D6
:103C0000EE50061902E1EE50071901E0026B4CEC90
:103C10001AF00901025112004CEC1AF0000C0101DB
:103C2000010E9ED8010E9CD8060E9AD8ABD8120E63
:103C300097D8230E95D8340E93D8560ECBD8800E35
:103C4000C9D8A0D89FD8316B2BEC19F00901196B9A
:103C50000C0E195D02E2A0D8FBD7BCC231F12BECEF
:103C600019F0BDC231F12BEC19F0BEC231F12BECD1
:103C700019F0BFC231F12BEC19F0C0C231F12BECBD
:103C800019F0C1C231F12BEC19F00901196B19516E
:103C9000106E116AD890115004E6CA0E105C000E26
:103CA000115802E279D8F3D70101630E59D8820E78
:103CB00057D8530E55D8630E53D8350E51D8010E30
:103CC000316F2BEC19F016C331F12BEC19F0030115
:103CD000160518E0085109110A110B1113E0010132
:103CE000360E7CD803C331F12BEC19F002C331F14D
:103CF0002BEC19F001C331F12BEC19F000C331F1B9
:103D00002BEC19F00101370E2BD8020E29D8010E29
:103D100027D8030E316F2BEC19F0030E0301165D4B
:103D200013E10101320E5AD808C331F12BEC19F01E
:103D300009C331F12BEC19F00AC331F12BEC19F066
:103D40000BC331F12BEC19F0010131692BEC19F0A7
:103D500090EF19F00101000E376F090EDCEF1EF035
:103D6000316F2BEC19F00101120026D8010112006D
:103D7000030114510301645D106E65510301155573
:103D8000116E1200316B2BEC19F00101120064C3AB
:103D900014F365C315F312000101316B2BEC19F01C
:103DA0000901192B120076C32FF11EEF19F0D2DF93
:103DB000040E0901005D1200386FFEEF19F0166F56
:103DC0002EDFE5DF03011200D3DF900E105CFF0E43
:103DD00011581200C5DFD6DFC2EF1EF0C1DF040E9E
:0E3DE000316F2BEF19F0B6DF0901012B120035
:023DEE000001D2
:103DF000F35101E112000001290EF16F5F0EF26F25
:103E0000FCEC33F00001390EF16F5D0EF26FFCEC4B
:103E100033F0F3C0B4F90901B451000814E2B4510D
:103E2000070B05E100012E0EED6F9DEC33F027DA54
:103E300002E057D908D0320EE66E97EC35F0E55225
:103E40000901B407E8D744EF21F03CDAE7D9010EC5
:103E5000E926000EEA22E2D9020EE926000EEA2245
:103E6000DDD9030EE926000EEA2255EF21F0090103
:103E7000016B05DAFEE08DEC33F00901006F0D0EE9
:103E8000005D17E00A0E005D14E0012B0001F6C092
:103E9000E9FFF7C0EAFFF62B000EF72300C9EFFF9A
:103EA000F6C0E9FFF7C0EAFFEF6AF851F80700092A
:103EB000E0E1090101511200F9C001F9FAC002F96B
:103EC0000901036BF9C0E9FFFAC0EAFFEFCF00F97F
:103ED000EF5021E02E0E0901005D11E10001F9C053
:103EE000E9FFFAC0EAFFF92B000EFA23EF6AAFD917
:103EF000032BD1D9F9C001F9FAC002F907D0300E6D
:103F0000005D03E30051390801E2000C0001F92BC8
:103F1000000EFA23D7D79BD9BED9030E0901035D42
:103F200001E0000C010CABD9FEE08DEC33F009018F
:103F3000006F310E005D05E3390E005D02E20051B5
:103F40001200390CA1D9300E0001FD5DFF0FE96EA2
:103F5000EA6AD890E936EA362D0EE926030EEA22FF
:103F6000EECFF1F0EDCFF2F0FCEC33F00001FD51BB
:103F7000380A01E1B5D00F0A01E1B0D0010A01E130
:103F8000A1D0030A01E197D0010A54E0070A4BE0EF
:103F9000010A42E0030A01E012000201330ED66F6B
:103FA000A6EC32F00901A16F0201340ED66FA6EC27
:103FB00032F00901A26F870EE66E090EE66EA1C906
:103FC000E6FFA2C9E6FF87D9870EEF6F090EF06FF3
:103FD000EBEC33F029D9000947E0870EE66E090EB5
:103FE000E66E75EC2CF0E552E552F3CFA1F9F4CF73
:103FF000A2F9F3CFA8FF0201330ED76FB0EC32F075
:10400000A2C9A8FF0201340ED76FB0EC32F0A2C9EA
:10401000C0F2A1C9C1F212000901B80E9F6F020ED1
:10402000A06FA36B0ED00901C60E9F6F020EA06F8A
:104030000E0E06D00901C20E9F6F020EA06F0A0E6F
:10404000A36F9FC9F4F0A0C9F5F0FFDEEDD8000121
:104050009B0EFB6F090EFC6F0001870EF96F090EB6
:10406000FA6F2ADF00090BE10001DF0EF16F5E0E2F
:10407000F26FFCEC33F003D9FEE08DEF33F09FC913
:10408000E9FFA0C9EAFF9BC9EEFF9CC9EEFF9DC9ED
:10409000EEFF9EC9EEFF9BC9A8FFEAD89CC9A8FF06
:1040A000E7D89DC9A8FFE4D89EC9A8FF0901A3517C
:1040B000A32B020110D00201160ED66FA6EC32F02F
:1040C000010906D00201160ED66FA6EC32F0FE0BE7
:1040D000A86E0201160ED76FB0EF32F086EF20F017
:1040E00012000001720EF16F5D0EF26FFCEC33F006
:1040F0001ADF0901B56F390EB55D03E0B5C9FDF0F2
:1041000021DF380E0901B55DECE112000901006BF9
:10411000026B0FEC25F064C385F965C386F90901CC
:1041200085510301645D106E655109018655116E5C
:10413000320E105C000E115809E364C385F965C3A3
:1041400086F90001150EED6F9DEC33F098D8E7E08D
:104150000901025162E193D8FBE08DEC33F00901D3
:10416000016F0051030A20E0010A1BE0030A14E07A
:10417000010502E1010E16D0040E015D09E158ECC3
:1041800025F00001060E9BD80901010E026FE0D751
:104190000001150E94D8DCD7060E046F036B020ED7
:1041A00001D0030E006FD4D70351032BEA6A050F29
:1041B000E96E090EEA2201C9EFFF0351106E116A80
:1041C0001134C6E210508008000E1154C1E2060EF0
:1041D000046F016B0151106E116AD890115004E602
:1041E000800E105C000E11580DE20151EA6A050FB5
:1041F000E96E090EEA22EFCF45F227EC25F009011E
:10420000012BE8D70201376B7FEC24F004C9EDF0F5
:104210009DEC33F00901006B9BD7010C46D80001DF
:104220002E0E4DD862EF21F00001290E48D8000172
:104230003A0E45D80001200E42D80001140EF86F46
:104240000001870EF66F090EF76F37EF1FF001C9F7
:10425000E6FF02C9E6FF75EC2CF0E552E552F3509B
:10426000E66EFBC010F0FCC011F009010351120012
:104270000901A351A32B0201D76FB0EF32F0000167
:10428000EA510001EB5D120000010D0E18D800018B
:104290000A0E5FEF21F00F011024E96E000E1120CD
:1042A000EA6EE552E750EF6E1200EF50E66EE66AF6
:1042B00012D8000EEF6F090EF06FEBEF33F0ED6FD9
:1042C0009DEF33F0000EE66E090EE66EF4C0E9FFD6
:1042D000F5C0EAFF1200EAEC2CF0E552E552E55297
:0642E000E552000112008E
:0A42E600150E01014F6F506B6EECD6
:1042F00000F00101936F976BC56B926B140E956F75
:10430000966B120093C155F12CEC01F0000907E106
:104310000101C56B070E996F976B926BA6D093C185
:1043200069F144EC03F0000934E020DA0101700E79
:10433000626F090E636F93C161F1B9EC02F000097D
:104340000EE01F0E0101C55DF1E2C551C52BEA6A01
:10435000A40FE96E010EEA2270C9EFFFE7D793C1FF
:1043600060F19BEC02F00A0E0901705D26E101018B
:10437000C551EA6AA40FE96E010EEA22EF6AC56B25
:104380009BD9C6C1D8F1C7C1D9F15DD90101996FD7
:1043900014D00101975111E0D5510301645D106EF5
:1043A00065510101D655116E500E105C460E115824
:1043B00004E3DCD9020E996F976F01019751020A4D
:1043C0003EE0070A0DE0040A06E0010A54E19A6B98
:1043D000CDD9010E976FBED94EE00101050E976F42
:1043E000B9D92DE09AC1E9FFEA6AE9BEEA68D89036
:1043F000E936EA36A20EE926020EEA22EECF71F97C
:10440000EDCF72F9090171C9F6FF72C9F7FF712B7F
:10441000000E72230800F5CF70F9F55007E070C95F
:104420005AF193C159F1F2EC01F0ECD793C157F175
:1044300075EC01F001010B0E9A6F020E976F070EDB
:104440000101995D18E099C1D7F116D800090FE074
:104450000B0E01019A5D02E0050E04D0020E995D7B
:1044600002E1010E976F070E996F986B010C0B0E0E
:1044700001019A5DB3E1010C0101D751050A51E038
:10448000060A4DE0070A34E0060A30E0030A18E0A5
:10449000010A51E192819293010E9A6F090EE66E24
:1044A000E66AC8C1E6FFC9C1E6FF9B0EE66E010ED3
:1044B000E66E45EC32F0106E060EE15E1050010C17
:1044C00092A112D0C8C16FF3C9C170F303019B0E52
:1044D0006D6F010E6E6F75EC30F0000904E00101A4
:1044E0009283020E29D00101060E26D09EEF22F003
:1044F000D0C1E6FFD1C1E6FF75EC2CF0E552E552E4
:10450000F3CF96F1D2C1E6FFD3C1E6FF75EC2CF0F4
:10451000E552E552F3CF95F101010A0E0DD0C7EF38
:1045200022F00A0E9A6FFE0E945D07E094C156F1D8
:1045300035EC01F0010C050E9A6F010C0101985148
:10454000030A18E0020A0FE0010A20E1020E985D5A
:1045500002E158EC25F0FE0E0101945D06E010D951
:104560000101010E05D0FCD811E10101030E9A6F83
:10457000986F000CEFD80AE093C155F12CEC01F0D4
:10458000000904E093C156F135EC01F0000C010183
:104590009851020A2EE0030A21E0010A53E192B386
:1045A00002D0060E4DD0070E9A6F95C153F196C1F9
:1045B00054F19351220DF3CFE9FFF4CFEAFF000E3F
:1045C000E9260A0EEA22EE52E9CF51F1EACF52F182
:1045D000AAEC00F00101946F010E09D0C1D832E0BD
:1045E000020131A12FD00FEC25F00101020E986FCE
:1045F000000C94C169F144EC03F000091AE0B6D84C
:104600000101730E626F090E636F94C161F1B9EC21
:1046100002F0000905E073C945F227EC25F0F0D758
:104620000201376B7FEC24F094C160F19BEC02F047
:10463000000C96D807E1A4D80101FE0E946F090E74
:104640009A6F010C000C0901006B060EE76E001951
:10465000E8AE02D0E73402D0E750005D2CE2040E51
:10466000E66EE66A00C9E9FFEA6AE9BEEA68D89040
:10467000E936EA36960EE926020EEA22EECF10F06F
:10468000EFCF11F0126A10C0E6FF11C0E6FF12C0B2
:10469000E6FFD8C1E6FFD9C1E6FF9BEC31F0136E0F
:1046A000070EE15E1350000903E1090100511200F9
:1046B0000901002BCAD7060C0901036BA40E006F79
:1046C000010E016F58D8EF50200804E1002B000EB6
:1046D0000123F8D700C9C6F101C9C7F10101010ED4
:1046E000D46F49D8EFCF02F9EF5033E009010351FD
:1046F000010A16E0010A29E1200E025D03E02C0EFA
:10470000025D05E138D8EF6A010E036F1ED00D0E71
:10471000025D03E00A0E025D18E12DD8EF6A15D0A4
:10472000200E025D12E00101D451D42BE96EEA6A39
:10473000D890E936EA36C60EE926010EEA2200C90B
:10474000EEFF01C9EDFF0901036B002B000E0123F1
:10475000C8D7120093C158F1D9EC01F0000912003A
:1047600094C155F12CEC01F00009120064C3D5F19D
:1047700065C3D6F1120000C9E9FF01C9EAFF1200C2
:0C47800058EC25F094C156F135EF01F023
:04478C000201306B8B
:10479000010E316F0301180E3D6F9BEC30F00901E3
:1047A000006B060E005D05E2005191D9EF6A002B07
:1047B000F8D7010C0901FE0E026F020131A1FE0CB7
:1047C0000901016B060E015D0AE2015180D9EF502B
:1047D000010B03E101C902F902D0012BF3D7FE0E50
:1047E000025D01E1FE0C450E036F046B056B33C2E5
:1047F000E9FF34C2EAFFEF5001E1FF0C33C2E6FFEC
:1048000034C2E6FF73EC32F0E552E552F3CF33F2F7
:10481000F4CF34F203C942F304C943F367D904E087
:104820000901FE0E026F5ED025EC31F00901006F28
:1048300000AF02D0026956D0016B0C0E015D21E27F
:1048400025EC31F00901006F01510201EA6A3325BC
:10485000E96E3451EA22EF500901005D06E0120EC4
:104860000327000E042305230CD0005108E10901A1
:10487000012B0C0E015D05E225EC31F0F8D7012B80
:10488000DCD70C0E015D2BE10251080DF3CF06F9C8
:10489000F4CF07F9000E0627020E072333D9010EC5
:1048A000EF6E30D9EB6A020EEB6A25EC31F0E66E62
:1048B00029D9030E03D9030E2AD9010EFFD8030EFE
:1048C00026D9020EFBD8060EF9D8060E20D9010E05
:1048D0001ED9E552E750EF6E0201302B03D02FECCA
:1048E00031F098D72FEC31F009010251120036C295
:1048F00037F205D802013651EAD8EF6A12000201F8
:104900003751080DF3CFAFF9F4CFB0F9000E09011C
:10491000AF27020EB023F1D8EF50020B03E02FECCB
:1049200031F00DD0EAD8EF50040B09E01BEC31F068
:104930000301A00E4B6F6AEC31F00009F9E1F90EAA
:10494000DCD8E850EF160201319312000201385111
:10495000080DF3CF01F9F4CF02F9000E0901012788
:10496000020E02239F0E106EBCD8E850EF16B9D885
:10497000EF50010B25E0B5D8EF50020B24E1020106
:1049800031B31ED0AED8EE52EECF13F0EFCF14F00D
:10499000156AA7D8030EBBD8EE501324106EEE5044
:1049A0001420116EEE501520126E10C042F311C08B
:1049B00043F39CD805E195D8EF820201318303D0FF
:1049C00090D8EF8A000C25EC31F00901006F89D8EE
:1049D000EE52EE2A000EED22EECF10F0EDCF11F0E8
:1049E00080D8060E94D8EECF12F0EFCF13F000016E
:1049F0001250101805E11350111802E172D8EF8C13
:104A0000090100511200010C010C12001200F36A9E
:104A1000F46A1200056A066A076A1200000C0201B5
:104A200031A1000C0901AF6B060EAF5D08E2AF517A
:104A30004ED8EF50010B01E0000CAF2BF5D702016F
:104A4000010E006F400E036F046B056B010C090132
:104A5000000EB16F020EB26F020100A506D0400E2B
:104A6000325D03E30201376B4ADF020100B515D066
:104A700031A302D0008B000C03C23FF304C240F309
:104A80000301A00E3E6FA4EC30F0000905E1020125
:104A900000853183326B01D0000C45C244F307EC32
:104AA00031F00201322B032B000E04230523010CED
:104AB0000201376B24DF0201006B010C28D8E5529C
:104AC000E750EF6E25EC31F0E66E82EF25F0080D31
:104AD000F3CFE9FFF4CFEAFF000EE926020EEA2247
:104AE000120001C9E9FF02C9EAFF12000301A00E8A
:104AF000416FDAEC30F000091200AFC9E9FFB0C92C
:104B0000EAFF120006C9E9FF07C9EAFF1200E92619
:064B1000000EEA22120073
:0A4B1600D9C2F3FFD8C2F4FF120069
:104B2000DAC201F9DBC202F9DCC203F9DDC204F921
:104B30000901010E056F090E066F05C9E9FFEA6E4E
:104B4000030E9AD9EF50E66E030E90D900C9EFFF1D
:104B500084D9020E91D9010E85D9EF50E66E7DD928
:104B6000020E84D9010E7ED900C9EFFF01C904F0FD
:104B700002C905F003C906F004C907F012000901D3
:104B8000406B416B426B436BDEC23EF9DFC23FF9C3
:104B9000E0C23CF9E1C23DF9D8903D333C333CC919
:104BA00010F03DC911F03C07000E3D5B1050111094
:104BB00018E03EC9E9FF3FC9EAFF020E3E27000E9A
:104BC0003F23EECF10F0EFCF11F00001105009019C
:104BD00040270001115009014123000E42234323C5
:104BE000DED70201E051010B0EE03EC9E9FF3FC9EB
:104BF000EAFFEFCF10F00001105009014027000E2E
:104C000041234223432309014251431109E040510A
:104C10004225406F41514321416F426B436BF3D7B3
:104C200040C910F041C911F0101E111E10C0F3FF51
:104C300011C0F4FF12000901010E006F016B026B3D
:104C40000201E251E3114EE0400EE25D000EE35935
:104C500004E3400E106E116A04D0E2C210F0E3C209
:104C600011F010C005F9090110500201576F586B7F
:104C70000201060E556F090E566F27EC0DF0090163
:104C80000551106E116A10500201E25F1150E35B92
:104C90000901046B0551045DD3E20451EA6A060F71
:104CA000E96E090EEA22EFCF03F900510AE1035140
:104CB0000125016F0351015D0DE2022B0BE1012B78
:104CC00009D003510225026F0351025D03E2012B5B
:104CD00001E1022B005102E0000E01D0010E006F35
:104CE000042BD8D70901021D026F011DF36E02C902
:104CF000F4FF12000201E451390805E3300EE45DCF
:104D000002E3300E0FD0E451460805E3410EE45DA6
:104D100002E3370E07D0E451660806E3610EE45D56
:104D200003E3570EE45D1200FF0C010E0201EA6A74
:104D3000E525E96EE651EA22EFCFE4F2DBDF090177
:104D4000236FE5C2E9FFE6C2EAFFEFCFE4F2D2DF6C
:104D50000901246FFF0E235D03E0FF0E245D01E1D6
:104D6000000C2439F00B2311E7C2E9FFE8C2EAFF87
:104D7000EF6E010C0901236BA6B2FED72F0EA6160B
:104D8000A6840201EBC2E9FFECC2EAFFEB2B000EA6
:104D9000EC23EF50A86E0901232B0201ED5109010C
:104DA000D880235501E2A86AEAC210F0116A1050B7
:104DB000AA6E0201E9C210F0EAC211F0E92B000E5E
:104DC000EA231050A96E550EA76EAA0EA76EA682F2
:104DD0000000A6B2FED7A850D4E1A6940901235141
:104DE00000D01200F1C210F01050AA6EF0C2A9FF5C
:104DF0003F0EA6160201EEC2E9FFEFC2EAFFEE2B5C
:104E0000000EEF23EFCF1CF9A680A85009011C5D0E
:104E100001E0010C1C5101E1000CA92AEBE1AA2AD6
:104E2000E9D7F2C202F9F3C203F90901006B016B81
:104E30000201F4510901005D0201F5510901015916
:104E40000BE202C9E9FF03C9EAFF022B000E0323AC
:104E5000EF6A002B0123ECD7120005C9E9FF06C950
:104E6000EAFF1200E926000EEA221200FBDFE552FB
:104E7000E750EF6E2DEF27F0F5DFEFCF00F92DEFC4
:024E800027F019
:0E4E8200140E0201576F586B0201080E556F97
:104E9000090E566F27EC0DF0F00E090108154008B9
:104EA00001E0A1D00F0E0815040DF350106E116A29
:104EB000140E105E000E115A10C01CF91050140888
:104EC00001E291D01C5100080BE21C510201576F06
:104ED000586B02011D0E556F090E566F27EC0DF031
:104EE00012C900F913C901F90901126B136B140EF1
:104EF00016D9080EDE6F090EDF6FBFEC25F0F3CF79
:104F000004F9F4CF05F90901041F051F1C5100081D
:104F100010E21C5104D91D0EDE6F090EDF6FBFECCD
:104F200025F0F3CF06F9F4CF07F90901061F071F93
:104F300002D0066B076B040EF2D8040EDE6F090E6A
:104F4000DF6FBFEC25F0F3CF02F9F4CF03F90301D3
:104F5000080E596F090E5A6FB5D809010251001990
:104F600042E1035101193FE1F00E081540083BE111
:104F700003014C514D110CE04CC3E9FF4DC3EAFF56
:104F800018C9EEFF19C9EEFF1AC9EEFF1BC9EEFFE3
:104F90004EC3E9FF4FC3EAFF060EDBD814C9EEFF8C
:104FA00015C9EEFF16C9EEFF17C9EEFF50C3E9FFA2
:104FB00051C3EAFF11C9EFFF09011C51126E136AB8
:104FC00012500A5D106E13500B59116E140E105EC4
:104FD000000E115A52C3E9FF53C3EAFF10C0EEFF9F
:104FE00011C0EDFF010C97EC0DF0000C0901450E0E
:104FF000286F296B140E0301572509012A6F000E33
:105000000301582109012B6F0101FD2B000EFE2326
:10501000FDC12CF9FEC12DF909012E6B400E2F6F39
:10502000640E306F56C331F9326B336BB8C234F94A
:10503000B9C235F9BAC236F9BBC237F954C3E9FF70
:1050400055C3EAFF060E85D8EECF38F9EECF39F911
:10505000EECF3AF9EFCF3BF90301280E596F090E55
:105060005A6F30D8140E5BD8280EDE6F090EDF6F32
:10507000BFEC25F0F3CF32F9F4CF33F9140E03016E
:1050800057250201626F000E030158210201636F70
:105090000201616B54C3E9FF55C3EAFF54C35FF2D9
:1050A00055C360F28FEC0EF0140E0201536F546B77
:1050B0000201280E516F090E526F9CEC0BF0F36A3F
:1050C000F46A120027D8020E35D8020E38D8020E24
:1050D0002BD8020E39D8040E2DD8040E30D8040E69
:1050E00023D8040E31D8060E25D8060E28D8060E71
:1050F0001BD8060E29D80A0E1DD80A0E20D80A0E73
:1051000013D80A0E03D83CC9EFFF120022D8010EB3
:10511000A9EF28F059C3E9FF5AC3EAFF12000201C0
:10512000E06FE16B0201120014D8E552E750EF6E18
:105130008AEF28F00ED8EFCF3CF98AEF28F0E6DFAF
:10514000EF50E66E8AEF28F0E1DF3CC9EFFF8AEF0F
:0A51500028F0E926000EEA22120002
:06515A00485454502F31AF
:105160002E3020353033200D0A0D0A5365727669D2
:10517000636520556E617661696C61626C650D0ACC
:10518000000D0A0D0A00485454502F312E302032A1
:105190003030204F4B0D0A436F6E74656E742D7462
:1051A0007970653A2000485454502F312E30203405
:1051B0003034204E6F7420666F756E640D0A0D0AD0
:1051C0004E6F7420666F756E642E0D0A00617564F3
:1051D000696F2F782D77617665006170706C6963F7
:1051E0006174696F6E2F6A6176612D61726368699F
:1051F000766500696D6167652F6A70656700696D26
:105200006167652F67696600746578742F6A6176D7
:105210006173637269707400746578742F6373735B
:10522000006170706C69636174696F6E2F6A61767A
:10523000612D766D00746578742F68746D6C0074E0
:105240006578742F706C61696E00477565737400C2
:105250004E6F0053757065722055736572000D0AAC
:105260004E6F772072756E6E696E67206170706C1C
:1052700069636174696F6E2E2E2E000D0A5265618E
:10528000647920746F20646F776E6C6F6164204660
:10529000696C652053797374656D20496D6167652C
:1052A000202D2055736520586D6F64656D207072D8
:1052B0006F746F636F6C2E0D0A000D0A44484350E3
:1052C000202620495020476C65616E696E67206416
:1052D000697361626C65642E0D0A000D0A444843CF
:1052E00050202620495020476C65616E696E67200A
:1052F000656E61626C65642E0D0A000D0A44656678
:1053000061756C74205375626E6574204D61736BAA
:105310002028000D0A44656661756C74204761742D
:105320006577617920416464726573732028000D8C
:105330000A44656661756C7420495020416464724A
:105340006573732028000D0A53657269616C204EE5
:10535000756D626572202800323030206F6B0D0A47
:1053600000323236205472616E7366657220436F6C
:105370006D706C6574650D0A0031323520446F6EB6
:10538000652E0D0A00313530205472616E736665EA
:105390007272696E6720646174612E2E2E0D0A0090
:1053A000353330204C6F67696E2072657175697294
:1053B00065640D0A00353032204E6F7420696D70BF
:1053C0006C656D656E7465640D0A00353030200DB6
:1053D0000A00323231204279650D0A003233302022
:1053E0004C6F6767656420696E0D0A0033333120A6
:1053F00050617373776F726420726571756972653D
:10540000640D0A003232302052656164790D0A0061
:1054100041424F5200504F52540053544F5200518A
:0E542000554954005041535300555345520016
:02542E001C0E52
:105430000201576F586B0201000E556F090E566F2F
:1054400027EC0DF097EC0DF00301000E626F090ED2
:10545000636FF5D80901010E001912E1015110E145
:105460000451106E116A060E10180AE1115008E17D
:105470000551126E136A040E121801E1135001E077
:10548000000C020E061905E1075103E106D9EF6A87
:105490000DD0010E061906E1075104E1010EFDD8F9
:1054A000EF6E04D0020EF9D8EF6E000C0201B85175
:1054B0000901185D2EE10201B9510901195D29E1C7
:1054C0000201BA5109011A5D24E10201BB5109012F
:1054D0001B5D1FE15BC3E9FF5CC3EAFF08C9EEFF88
:1054E00009C9EEFF0AC9EEFF0BC9EEFF0CC9EEFFBA
:1054F0000DC9EEFF5BC3E9FF5CC3EAFF060ED7D818
:105500000EC9EEFF0FC9EEFF10C9EEFF11C9EEFF85
:10551000010C000C010E0901006F016B026B080EFB
:10552000036F060E046F040E056F030161050BE1A6
:10553000010E0901066F076B126913691469156979
:105540001669176914D0020E0901066F076B5FC355
:10555000E9FF60C3EAFFEECF12F9EECF13F9EECF09
:1055600014F9EECF15F9EECF16F9EFCF17F9BCC24B
:1055700008F9BDC209F9BEC20AF9BFC20BF9C0C21F
:105580000CF9C1C20DF9B8C20EF9B9C20FF9BAC20D
:1055900010F9BBC211F97AD8EF500E190201C215E9
:1055A0001BE174D8010E83D8EF5009010F190201D5
:1055B000C31512E16BD8020E7AD8EF500901101909
:1055C0000201C41509E162D8030E71D8EF50090138
:1055D00011190201C51509E0C6C218F9C7C219F9A7
:1055E000C8C21AF9C9C21BF909D050D8EECF18F9B0
:1055F000EECF19F9EECF1AF9EFCF1BF90301000E28
:10560000626F090E636F1BD81C0E0201626F636B21
:105610000201060E616F0201120E5F6F090E606FCC
:105620008FEC0EF01C0E0201536F546B0201000E42
:10563000516F090E526F9CEC0BF0E6EF0EF032D872
:1056400019D8F3CFEEFF11C0EDFF2CD8020E2FD8E2
:1056500011D8020EF3CFEBFF030E11C0EBFF22D8DF
:10566000060E25D807D8060EF3CFEBFF070E11C0A4
:10567000EBFF1200EECFD8F2EDCFD9F28BEC25F094
:10568000F3CF10F0F4CF11F052EF2BF05FC3E9FF2E
:1056900060C3EAFF060E57EF2BF05DC3E9FF5EC360
:1056A000EAFF120062C3E9FF63C3EAFF1200E926C2
:0656B000000EEA221200C8
:0A56B6000B01BD6BBE815EEC0AF033
:1056C0000EEC34F0C4EC18F03AEF00F00901010ED2
:1056D000B46F0901B45101E1FDD0B46B0B01BD51B0
:1056E000040A01E1D7D0070A01E1A1D0050A01E1CE
:1056F00087D0010A72E0050A3FE0070A36E0050A92
:1057000002E0010AE6E10201B30E5D6F090E5E6F71
:105710000201BF0E5B6F0B0E5C6FDCEC0DF000093D
:1057200015E10201160ED66FA6EC32F0010BD1E0A6
:10573000CEEC0DF00009CDE10201B86BB96BBA6B8C
:10574000BB6B0B01BE8123EC1CF0C3D70901010E1A
:10575000B46FB35103E10B01020E39D0060EB35DF5
:1057600001E095D00B01050E32D00901B46B1BECA2
:1057700034F00009AEE0ABD00301C90E526F0B0E3E
:10578000536F0301B30E506F090E516F0301BF0E2B
:105790004E6F0B0E4F6F0301AF0E4C6F090E4D6F26
:1057A00041EC27F0000916E00901010EB46FB305C2
:1057B00003E10B01030E0BD0060EB35D03E10B01F9
:1057C000060E05D0110EB35D04E10B01070EBD6F8F
:1057D00080D7B46B97EC0DF07AD0C9CB41F1CACB2E
:1057E00042F10101AF0E3F6F090E406F0101BF0E84
:1057F0003D6F0B0E3E6F54EC1AF0000915E012D00D
:10580000C9CB6EF1CACB6FF10101AF0E6C6F090EFF
:105810006D6F0101BF0E6A6F0B0E6B6F2DEC04F004
:10582000000902E00B01BD6B0901B46B52D7BD6BDF
:10583000290ED880C955000ECA5529E30301ED0E83
:105840001F6F0B0E206F0301EB0E1D6F0B0E1E6FF3
:105850000301C90E1B6F0B0E1C6F0301CB0E196FDA
:105860000B0E1A6F0301B30E176F090E186F84EC3D
:105870002DF000090AE0080E0901B35D06E1010EF2
:10588000B46F0B01040EBD6F02D00B01BD6B97EC22
:105890000DF01FD74CEC0BF0000901E11AD7EDCB4E
:1058A00029F3EECB2AF3EBCB27F3ECCB28F3C9CBD0
:1058B00026F30301CB0E246F0B0E256F0301236B20
:1058C0000301BF0E216F0B0E226FFEEC2DF00B01BA
:1058D000BD6BFFD651EC03F031EC1CF0030177A156
:0A58E00002D00B01BE9133EF0BF074
:0658EA00FF0EE3CFEAFF10
:1058F000E552FF0EE3CFE9FFE552E66AE66AD9CF4B
:10590000E6FFDACFE6FFFC0EE124D96EFF0EE220BF
:10591000DA6EE66AE66AE66A200EEF5C06E0090ED9
:10592000EF5C03E0EF6603D03FD0EE50F5D72D0ECD
:10593000EF5C03E1FF0EE32A03D02B0EEF5C01E1E5
:10594000EE502F0EEF6424D03A0EEF6021D0D890A5
:10595000F90EE336FA0EE336FD0EDECFE3FFFE0E60
:10596000DDCFE3FFD890F90EE336FA0EE336D89098
:10597000F90EE336FA0EE336FD0EE350DE26FE0E98
:10598000E350DD22300EEE5CDE26000EDD22D9D79C
:10599000FF0EE3CFE8FFE85207E0F90EE31EE32A2B
:1059A000FA0ED8B4E306E31EE552E552E552FF0EC7
:1059B000E3CFDAFFE552FF0EE3CFD9FFE552E1CFA7
:1059C000E9FFE2CFEAFFED52ED52EECFF3FFEFCF6A
:1059D000F4FF1200D9CFE6FFDACFE6FFFA0EE3CFED
:1059E000D9FFFB0EE3CFDAFFFD0EE35209E72D0EE0
:1059F000DE6EFC0EE31EE32AFD0ED8B4E306E31EC2
:105A0000E652E652E652FD0EE124E76EFF0EE2207A
:105A1000E46EE652F70EE3CFE6FFF70EE3CFE6FFC4
:105A20005AEC2DF0F90EE124E96EFF0EE220EA6E49
:105A30004AEC2DF00AE147EC2DF009E14AEC2DF09B
:105A400008E147EC2DF007E108D055EC2DF050ECC3
:105A50002DF055EC2DF050EC2DF055EC2DF0DE6ACC
:105A6000F90EE126FF0EE222FF0EE3CFDAFFE55248
:105A7000FF0EE3CFD9FFE552FC0EE124E96EFF0EE5
:105A8000E220EA6EEECFF3FFEFCFF4FF1200EF3823
:105A90000F0B1200EF500F0B02E1EE52D8841200F0
:105AA000EF380F0B300FDE6E1200EE500F0B300F81
:105AB000DE6E1200FC0EE3CFE9FFFD0EE3CFEAFF3E
:105AC000100EE66EEE6AEE6AEF6AD890FD0EE336CF
:105AD000FE0EE336ED36ED36EF36FF0EE30609E057
:105AE0007BEC2DF0EE527BEC2DF0EE527BEC2DF0AA
:105AF000EDD7E56E1200030EEF24E8B6EF6E300E20
:085B0000EF24E8BEEF6E000C7B
:085B0800080E0201576F586BF3
:105B10000201000E556F090E566F27EC0DF002C9F9
:105B20002EF903C92FF90901026B036B080E02015C
:105B3000E06FE16B0201000EDE6F090EDF6FBFEC5C
:105B400025F0F3CF28F9F4CF29F90901281F291FDF
:105B5000080E106ED9D8E850EF5ED6D8EF5002018B
:105B6000576F586B19C355F21AC356F227EC0DF054
:105B7000CBD8EF500201E06FE16B19C3DEF21AC31C
:105B8000DFF2BFEC25F0F3CF2AF9F4CF2BF90901AE
:105B90002A1F2B1F040E0201E06FE16B0201280E89
:105BA000DE6F090EDF6FBFEC25F0F3CF2CF9F4CFD9
:105BB0002DF90301000E2B6F090E2C6F7AD817C335
:105BC000E9FF18C3EAFF00C9EFFF1DC3E9FF1EC3C9
:105BD000EAFF04C9EEFF05C9EDFF1FC3E9FF20C3BB
:105BE000EAFF06C9EEFF07C9EDFF09012E512C1986
:105BF00002E12F512D1901E0000C010C0901016B8C
:105C000023C300F9026B036B27C304F928C305F90A
:105C100029C306F92AC307F903012651E66EE66A8D
:105C200024C3E6FF25C3E6FF080EE66E090EE66E06
:105C3000BAEC31F0106E060EE15E10500301000E5A
:105C40002B6F090E2C6F35D8080E03012625020193
:105C5000E06FE16B000EE1230201000EDE6F090E22
:105C6000DF6FBFEC25F0F3CF02F9F4CF03F9080E94
:105C7000030126250301576F586B000E58230301BB
:105C8000010E566F21C354F322C355F3F6EC27F0EF
:105C9000080E030126250201536F546B000E542396
:105CA0000201000E516F090E526F9CEC0BF0E6EFF3
:105CB0000EF02FD8040E15D8040EF3CFEBFF050E0F
:105CC0001FD8060E0ED8060EF3CFEBFF070E18D81E
:105CD000020E07D8020EF3CFEBFF030E11C0EBFF4D
:105CE0001200E926000EEA22EECFD8F2EDCFD9F26B
:105CF0008BEC25F0F3CF10F0F4CF11F089EF2EF0FC
:105D000011C0EBFF89EF2EF01BC3E9FF1CC3EAFFB4
:0C5D100012002BC3E9FF2CC3EAFF1200B5
:045D1C004D6F6474EF
:105D2000726F6E6978205443502F4950205374612C
:105D3000636B2056332E3033000D0A507265737337
:105D400020616E79206B657920666F7220436F6EDB
:105D500066696775726174696F6E206D656E752E08
:105D600000444843502F476C65616E696E672E2E64
:105D70002E000D0A0D0A0D4D78576562537276722A
:105D80002044656D6F204170706C69636174696F48
:105D90006E2076312E3020284D6F6474726F6E69DC
:105DA00078205443502F495020537461636B205620
:105DB000332E30332C204D6172203036203230307B
:105DC00036290D0A0D0A09313A204368616E67656C
:105DD00020426F6172642073657269616C206E7518
:105DE0006D6265722E0D0A09323A204368616E6752
:105DF000652064656661756C742049502061646437
:105E0000726573732E0D0A09333A204368616E6719
:105E1000652064656661756C74206761746577617F
:105E20007920616464726573732E0D0A09343A2017
:105E30004368616E67652064656661756C74207384
:105E400075626E6574206D61736B2E0D0A09353AAB
:105E500020456E61626C65204448435020262049ED
:105E60005020476C65616E696E672E0D0A09363ADF
:105E70002044697361626C652044484350202620A9
:105E8000495020476C65616E696E672E0D0A0937AF
:105E90003A20446F776E6C6F61642046696C6520B0
:105EA00053797374656D20496D6167652E0D0A091C
:105EB000383A2053617665202620517569742E0D7D
:105EC0000A0D0A456E7465722061206D656E75203D
:105ED00063686F6963652028312D38293A20000DE9
:105EE0000A496E76616C696420696E7075742072FF
:105EF00065636569766564202D20496E7075742030
:105F000069676E6F7265642E0D0A50726573732037
:105F1000616E79206B657920746F20636F6E746990
:0E5F20006E75652E2E2E0D0A001B5B324A0098
:025F2E00DACFC8
:105F3000E4FFE2CFDAFFE9CFE4FFEACFE4FFF6CFF8
:105F4000E4FFF7CFE4FFF5CFE4FFF3CFE4FFF4CFB6
:105F5000E4FFFACFE4FF00EE00F0100EE80403E3E4
:105F6000EECFE4FFFBD700EE10F0080EE80403E3E9
:105F7000EECFE4FFFBD7E652F2A414D09E0ED76E0C
:105F8000580ED66E0301642B000E6523662367232B
:105F900003016A0706E1640E6A6F0301682B000EB5
:105FA0006923F2949E50200B05E09D50200B02E0E7
:105FB00060EC33F09E50100B05E09D50100B02E09A
:105FC00076EC33F0E55200EE17F0080EE80403E338
:105FD000E5CFEDFFFBD700EE0FF0100EE80403E372
:105FE000E5CFEDFFFBD7E5CFFAFFE5CFF4FFE5CF37
:105FF000F3FFE5CFF5FFE5CFF7FFE5CFF6FFE5CF00
:10600000EAFFE5CFE9FFE5CFDAFF110088D8C4EC5D
:1060100035F0C6EC23F046EC14F04CEC33F088EC91
:1060200032F0C4EC32F055EC33F013EC33F02AECE0
:1060300033F03FEC33F00201140ED66FA6EC32F0D1
:106040000001F36FF7EC1EF05BEC2BF0B1EC0FF0FE
:1060500073EC21F00201160ED66FA6EC32F0010BA4
:1060600006E10001010EFE6F0301070E756F0201CC
:10607000150ED66FA6EC32F0020B0CE00001FF51BA
:106080000301645D106E320E105C04E364C3FFF024
:10609000939C8A7C66EC2BF051EC10F082EC21F0A2
:1060A00008D80001FE510301785DE1E078C3FEF0FD
:1060B000DED703016C2B0C0E6C5D01E36C6BC11C15
:1060C0000F0B6C5D0FE2C30EC2166C51040DF35042
:1060D000C212C280C282C2B2FED7030125D8C4CF89
:1060E000EFFF120021D8EF6A1200350E0201F06FA7
:1060F000F16B6DC3EEF26EC3EFF2F2EC26F0000925
:106100000DE13E0E0201F06FF16B6FC3EEF270C352
:10611000EFF2F2EC26F0000901E1010C000CF18E27
:10612000D56AF28EF28C12006C51EA6ACA0FE96EDF
:06613000020EEA2212003B
:0A6136003DC373F30301726B030114
:10614000080E716F7CEF35F03FC3AFF940C3B0F973
:10615000C750040B01E0010EE5D8FAE1C580C5B0D7
:10616000FED7A1B6010C3EC374F3E1D801E0010CE7
:10617000C750040B01E0010ED5D8FAE1C5BC19D017
:10618000B0C974F3D4D801E0010CC750040B01E08E
:10619000010EC8D8FAE1AFC974F3C9D801E0010C07
:1061A000C750040B01E0010EBDD8FAE1C5AC000CEC
:1061B000020C020C42C33FF343C340F341C33EF31E
:1061C000C3DF0901086FE85005E178D80901086FBD
:1061D000E85002E008511200C750040B01E0010E24
:1061E000A1D8FAE1C580C5B0FED7A1B6010C030164
:1061F00041290301746F9BD801E0010CC750040BC7
:1062000001E0010E8FD8FAE1C5AC000C020CC750BA
:10621000040B01E0010E86D8FAE144C374F387D879
:1062200001E0010CC750040B01E0010E7BD8FAE13C
:10623000C5AC000C020CC750040B01E0010E72D873
:10624000FAE1C584C5B4FED7000C8BEC35F0C5B6B9
:10625000FED7C59AC588C5B8FED7C95012008BECC9
:1062600035F0C5B6FED7C58AC588C5B8FED7C58482
:10627000C5B4FED7000C46C342F347C343F345C33E
:1062800041F398DF0901006FE85016E103014A511C
:106290004A0700090EE0D9DFE66E030148C3E9FFB3
:1062A00049C3EAFF482B000E4923E552E750EF6E41
:1062B000EDD7D5DF0901006F00511200C750040B64
:1062C00001E0010E2FD8FAE1C584C5B4FED7A1B60E
:1062D000010C000CC750040B01E0010E23D8FAE1B9
:1062E000C580C5B0FED7A1B6010C4BC374F31FD84F
:1062F00001E0010CC750040B01E0010E13D8FAE1D4
:10630000A1B6010CC5BC03D00901B36B03D00901D0
:10631000040EB36FC584C5B4FED7A1B6010C090144
:10632000B3511200106E1F0EC5141010120090EC25
:0663300035F00009120027
:0A633600FB0EE3CFF6FFFC0EE3CFF1
:10634000F7FFFD0EE3CFF8FFFE0EE3CFE9FFFF0EF0
:10635000E3CFEAFFF90EE35003E1FA0EE35009E060
:10636000F90EE30602E2FA0EE3060900F550EE5CD0
:10637000F1E01200D9CFE6FFDACFE6FFFA0EE3CF65
:10638000D9FFFB0EE3CFDAFFFC0EE3CFE9FFFD0EF2
:10639000E3CFEAFFE9CFF3FFEACFF4FFF80EE350D3
:1063A00003E1F90EE35008E0F80EE30602E2F90E0D
:1063B000E306DECFEEFFF2D7FF0EE3CFDAFFE552C2
:1063C000FF0EE3CFD9FFE5521200FB0EE3CFF6FF3D
:1063D000FC0EE3CFF7FFFD0EE3CFF8FFFE0EE3CF99
:1063E000E9FFFF0EE3CFEAFFE9CFF3FFEACFF4FFC7
:1063F000F90EE35003E1FA0EE35009E0F90EE3066B
:1064000002E2FA0EE3060900F5CFEEFFF1D7120023
:10641000FB0EE3CFF6FFFC0EE3CFF7FFFD0EE3CF5D
:10642000F8FFFE0EE3CFE9FFFF0EE3CFEAFF09001E
:10643000F550EF5C02E1EE66FAD71200FB0EE3CFF7
:10644000F6FFFC0EE3CFF7FFFD0EE3CFF8FFFE0EE5
:10645000E3CFE9FFFF0EE3CFEAFFE9CFF3FFEACF97
:10646000F4FF0900F5CFEFFFEE66FBD71200FE0E3A
:10647000E3CFE9FFFF0EE3CFEAFFF36AF46AEE52DF
:1064800003E0F34AF42AFBD71200D9CFE6FFDACFB4
:10649000E6FFFA0EE3CFD9FFFB0EE3CFDAFFFC0EE7
:1064A000E3CFE9FFFD0EE3CFEAFFE9CFF3FFEACF49
:1064B000F4FFF80EE35003E1F90EE3500BE0F80EA1
:1064C000E30602E2F90EE306DECFEFFFEE66F1D758
:1064D000DD52EFD7FF0EE3CFDAFFE552FF0EE3CF39
:1064E000D9FFE5521200FE0EE3CFE9FFFF0EE3CF26
:1064F000EAFFE9CFF3FFEACFF4FF610EEF5C05E6B8
:106500007B0EEF5C02E7DF0EEF16EE52F6E11200B3
:10651000AA6AA96A3F0EA6160901B80E006F020EFC
:10652000016FA950106E116A120E105C000E115806
:106530000CE2A68000C9E9FF01C9EAFF002B000EAA
:106540000123A8CFEFFFA92AECD71200D6C2A9FFDA
:10655000AA6AA6B2FED73F0EA616A680A8501200C1
:10656000D7C2A9FFAA6AA6B2FED72F0EA616A68486
:10657000550EA76EAA0EA76EA6820000A6B2FED781
:10658000A69400D012001200240EAC6E900EAB6EDA
:10659000080E7E6E02011F0E7CD8080A36E00F0A34
:1065A00032E0010A2AE0030A23E0010A1CE0070A9C
:1065B00015E0010A0EE0030A07E0010A28E10901DB
:1065C000340E1C6F820E1DD009018C0E1C6F200E24
:1065D00018D00901450E1C6F100E13D00901220EB0
:1065E0001C6F080E0ED00901100E1C6F040E09D08E
:1065F0000901080E1C6F020E04D00901030E1C6F66
:10660000010E1D6F08D0AC0E03D0560E01D0AC0E9B
:1066100009011C6F1D6B1CC9AFFF1DC910F0116A69
:1066200010507F6E12000201230E33D8926E0201C9
:10663000240E2FD8936E0201250E2BD8D809946E04
:106640000201280E26D8976E0201290E22D81009C1
:10665000986E120002012A0E1CD8896E02012B0EC0
:1066600018D88A6E02012C0E14D88B6E02012F0EE0
:1066700010D88E6E0201300E0CD88F6E12000201FF
:10668000310E07D8C16E0201320E03D87F0BC06EE7
:086690001200D66FA6EF32F0F4
:086698000001EC6BE06BE16B0B
:1066A000EA6BEB6B9D9A9D9812009D8A9D98120053
:1066B0000001E16BE1C0E0F0EB6BEBC0EAF012002F
:1066C000060EAB1402E0AB98AB889EAA0ED0000178
:1066D000EB51EA6AE20FE96E000EEA22AECFEFFF5D
:1066E000EB2B070EEB15EB6FF0D712000001E0511A
:1066F000E15D0DE0E051EA6A600FE96E000EEA220A
:10670000EF50AD6EE02B7F0EE015E06F12009D980C
:10671000120012000001EC5112000001EA51EA6A75
:10672000E20FE96E000EEA22EFCFAFF9EA2B070E77
:10673000EA15EA6F0901AF5112000001E129106E5C
:10674000116A7F0E1016000E11160001E051126E34
:10675000136A1250101802E11350111802E10400DC
:10676000ECD7F29E9DB805D0EDC0ADFF9D88F28EAE
:1067700011D00001E151EA6A600FE96E000EEA22D1
:10678000EDC0EFFF0001E12B7F0E0001E1150001DC
:10679000E16FF28E12000001EE519F0805E2EE3922
:1067A0000F0B0F0B570F04D0EE390F0B0F0B300FE1
:1067B0000001ED6FC2DF0F0E0001EE15090804E2C3
:1067C0000F0EEE15570F03D00F0EEE15300F000110
:1067D000ED6F9DEF33F00001EFC0E9FFF0C0EAFF7D
:1067E000EF2B000EF023EFCF08F9EF5004E008C9BB
:1067F000EDF0A3DFF0D712000001F1C0F6FFF2C008
:10680000F7FFF12B000EF2230800F5CF00F9F55049
:0C68100004E000C9EDF091DFEFD71200AA
:04681C000B01EF6B12
:10682000F069F169F269F369F469F569F66BF76B80
:10683000F86BF96B12000B01EF5129E10301260EF1
:106840005D6F090E5E6F03011C0E5B6F090E5C6FBE
:1068500017EC2AF000092CE00901265115E11CC9AA
:10686000F0FB1DC9F1FB1EC9F2FB1FC9F3FB20C9D8
:10687000F4FB21C9F5FB22C9F6FB23C9F7FB24C9A8
:10688000F8FB25C9F9FB010C0B01010EEF6F4CEC75
:106890000BF000090CE00301616B03011C0E5F6F3C
:1068A000090E606F8AEC2AF00B01EF6B010C000CF3
:1068B000010CFACBE9FFFBCBEAFFEECF22F9EECFDA
:1068C00023F9EECF24F9EFCF25F90301010E616F13
:1068D00003011C0E5F6F090E606F8AEF2AF0FCCB7C
:1068E000E9FFFDCBEAFF0B01F651EE1808E1F75185
:1068F000EE1805E1F851EE1802E1F951EE1814E036
:106900000201C6510B01F65D20E10201C7510B01E6
:10691000F75D1BE10201C8510B01F85D16E10201B0
:10692000C9510B01F95D11E1FECBE9FFFFCBEAFF95
:10693000F0CBEEFFF1CBEEFFF2CBEEFFF3CBEEFFB1
:0C694000F4CBEEFFF5CBEEFF010C000CD9
:04694C005458540047
:1069500048544D00434C4100435353004A530000F8
:1069600047494600434749004A5047004A415200C0
:1069700057415600545854005A5458005A4854002D
:106980005A434C005A4353005A4A530048545450F7
:106990002F312E3020323030204F4B00436F6E7439
:1069A000656E742D747970653A2000436F6E74655E
:1069B0006E742D456E636F64696E673A20677A69FD
:1069C000700D0A00457870697265733A20300D0ABF
:1069D0000043616368652D436F6E74726F6C3A207B
:1069E0006D61782D6167653D3330302C206D757396
:1069F000742D726576616C69646174650D0A004777
:106A0000455400494E4445582E48544D004C4F477C
:076A1000494E2E43474900E7
:086A18002A0EF66E000EF76E67
:106A2000000EF86E02010900F550FB6F0900F550E9
:106A3000FC6F03E1FB6701D03DD00900F550F66F14
:106A40000900F550F76F0900F550F86F09000900CB
:106A5000F550E96E0900F550EA6E090009000900D9
:106A6000F550F96F0900F550FA6F09000900F6CFEB
:106A7000FDF2F7CFFEF2F8CFFFF2F6C2F6FFF7C253
:106A8000F7FFF8C2F8FF0201F95302E1FA5307E0F9
:106A90000900F550EE6EF907F8E2FA07F9D7FDC2E2
:106AA000F6FFFEC2F7FFFFC2F8FF0201FB07000E70
:066AB000FC5BBFD71200E1
:0A6AB6004E6F7420496D706C656D21
:106AC000656E7465640073656C656374656400630A
:106AD0006865636B65640064697361626C6564001A
:106AE0003C212D2D002D2D3E006F6E006F6666003F
:076AF000557064617465003C
:086AF8003F0EC716C66AC56A0D
:106B000003017151C6127251C71294869488C68AC5
:106B100073C3C8FF1200C586C7A0FED7C9501200B4
:0E6B200074C3C9FFC6BEFF0CC7B0FED7000C81
:026B2E00FF0E58
:106B3000E3501D6EEF0E01D0F30EE76EE72E9EEFD1
:106B400035F00C0E1C6EE76AE72EA4EF35F01C2E14
:0C6B5000A3EF35F01D2E9CEF35F0120075
:046B5C00036A026A5C
:106B6000100EE76ED89006360736023603360B5005
:106B7000025C0C50035805E30B50025E0C50035AA4
:086B8000062AE72EF0D71200EF
:086B88000301646B656B666B91
:106B9000676B686B696B580ED66E9E0ED76E010ED2
:0A6BA000D56ED58EF284F28A120041
:066BAA00036A080EE76E0D
:106BB000D890073603360C50035C02E3036E072AB5
:066BC000E72EF7D71200DA
:0A6BC6001CEE00F02CEE00F0F86A5F
:0E6BD0000F9C0CEC35F006EC30F0FDD71200F7
:026BDE00FF0EA8
:106BE000E350E84E1200000000D000D000D0E82EA4
:046BF000FAD71200BE
:066BF40056322E3433007E
:066BFA0056332E3034007A
:106C000046532F531353FB52DB52BA527B525E5200
:026C1000000082
:026C1200000080
:0C6C14003F523552215218520852FE51D6
:106C20003552F351DA51CD513F523F523552215234
:0C6C300018520852A651865181515A5149
:046C3C00295424545F
:106C40001F541A54155410540454EC53DC53D253AB
:0E6C5000CB53B553A05385537953615358531A
:026C5E0000FF35
:026C6000000032
:020000040030CA
:0100010026D8
:0100020006F7
:010003000AF2
:010005008179
:010006008178
:010008000FE8
:01000900C036
:01000A000FE6
:01000B00E014
:01000C000FE4
:01000D0040B2
:0200000400F00A
:100000000A0100010004A3000000FF0000000A0133
:10001000000104012803000A0100010A0100010790
:10002000000700FFFFFFFFFFFFFF000000000000D0
:1000300000032E000061646D696E0000000070779F
:0700400000000000000000B9
:00000001FF
